:100000000C9492020C94D9020C94D9020C94D9024B
:100010000C94D9020C94D9020C94D9020C94D902F4
:100020000C94D9020C94D9020C94D3320C94A733BB
:100030000C94402D0C94D9020C94D9020C94D90242
:100040000C94D9020C94D9020C94D9020C94D902C4
:100050000C94D9020C94972D0C94D9020C94D902CB
:100060000C94D9020C94D9020C94D9020C94D902A4
:100070000C94D9020C94D9020C94D9020C94D90294
:100080000C94D9020C94D9020C94D9020C94D90284
:100090000C94D9020C94D9020C94D9020C94D90274
:1000A0000C94D9020C94D9020C94D9024C004A0049
:1000B0004D410000AC00AE00AB00A800005C520057
:1000C00001000000500051004F00145C01000100CD
:1000D0000100000001000100010001000100010019
:1000E000010000000100010001000100000000000B
:1000F000000000002A2B2800000000000000000083
:100100000000000000000029000000002C1E342028
:10011000212224342627252E362D3738271E1F204E
:100120002122232425263333362E37381F04050693
:100130000708090A0B0C0D0E0F10111213141516D7
:100140001718191A1B1C1D2F3130232D35040506D5
:100150000708090A0B0C0D0E0F10111213141516B7
:100160001718191A1B1C1D2F3130354C00000000C8
:10017000000000000000000000000000000000007F
:10018000000000000000000000000000000000006F
:100190007E0F00D4FFFFFFC700000078FD377A58BC
:1001A0005A000004E6D6B446020021011600000001
:1001B000742FE5A3E0011500B75D003D8889C654A2
:1001C00036C3174FE4E179499FE887A4B4005D91F5
:1001D0004E3B3ADA9DBBEF25E238845D3926FB3D84
:1001E000ABBFAAE8AD7817C97690D947B53BA71839
:1001F0002889C0AF97ACD626E3B357A87263830FA4
:100200004451E20DBE36E93DB09302107823636E8F
:10021000A6D869C7A65D78C782AF4E2EB70DA17E5E
:10022000BFD8FF1DB34BF8F40295C8A4CDC55A053D
:10023000BD73A8F14CA5DFEBE0C626385672A8FEC8
:10024000EA813CCCC2201ACBA1FB7A6776DD682F0D
:10025000B7B1C969187CE2BF40592B4C4BE264FA34
:100260009824D679DD31F8D6106E763514E4CE3D7B
:1002700019CC0000B1FC324AD944DD580001D30149
:1002800096020000FAF930F1B1C467FB02000000E9
:100290000004595AAA00A9001D011C010100010017
:1002A00001000100010001006704000002000200DB
:1002B0006304000003000100680400000400020061
:1002C0004D04ED2105000100690400000600020054
:1002D0004F04000007000200650400000800010050
:1002E0006A040000090002005104C8210A0002004B
:1002F0005304C8210B0002005504C8210C00020061
:100300005704C8210D0002005904C8210E00020044
:100310005B04C8210F0002005D04C8211000020028
:100320005F04C821110002006104C821120002000C
:100330006B040000130002006D0400001C03760033
:10034000690061006C003A0066003600340063000A
:100350003200620033006300000022034D006100A0
:10036000630072006F0042006F0061007200640061
:10037000200076002E0032002E0030000000140312
:100380004B006900770069004B0065006500620062
:10039000730000000403090409025B00030100A0CC
:1003A000FA09040000010301010009211101000103
:1003B0002240000705810308000A09040100020326
:1003C000000000092111010001222200070582031B
:1003D00020000107050303200001090402000103B6
:1003E00000000009211101000122BC00070584035F
:1003F00020000A1201000200000008514B124701C0
:1004000000010203010660FF0961A10109621500F4
:1004100026FF009520750881020963150026FF005C
:10042000952075089102C005010902A10185020904
:1004300001A100050919012905150025019505757A
:10044000018102950175038101050109300931150A
:1004500081257F95027508810609381581257F95CC
:100460000175088106050C0A38021581257F950162
:1004700075088106C0C005010980A1018503190125
:100480002AB700150126B700950175108100C00537
:100490000C0901A101850419012AA002150126A059
:1004A00002950175108100C005010906A1018505AD
:1004B000050719E029E71500250195087501810256
:1004C0000507190029EF1500250195F07501810236
:1004D0000508190129059505750191029501750316
:1004E0009101C005010906A101050719E029E715D9
:1004F00000250195087501810295017508810105A6
:1005000007190029FF150026FF00950675088100D0
:1005100005081901290595057501910295017503D5
:100520009101C00011241FBECFEFDAE0DEBFCDBFC6
:1005300004B603FE27C08091800490918104A091AD
:100540008204B09183048730904BA740B04BD1F424
:1005500010928004109281041092820410928304FD
:1005600014BE84B7877F84BF0FB6F894A895809196
:100570006000886180936000109260000FBEE0E030
:10058000F8E3099511E0A0E0B1E0E4E8FCE602C080
:1005900005900D92AC3AB107D9F724E0ACEAB1E08E
:1005A00001C01D92A038B207E1F70E9440150C94DB
:1005B0000E360C9400009C013A9521153F4150F5F0
:1005C000FC01EE27F170BC0166277270AC01442774
:1005D00054709C012227387094FF0EC080E1EF2BED
:1005E00009F480E0672B09F08062452B09F08064F4
:1005F000232B89F08068089581E0EF2B09F480E0D7
:10060000672B09F08260452B09F08460232B19F0D9
:100610008860089580E00895CF93DF93EC010E94F5
:10062000DB029E01205E31092830310510F0209751
:1006300039F40E94B3068C2FDF91CF910C94A8055A
:100640000E94C106F8CFCF93DF93EC010E943A06D7
:10065000CE010E94DB029E01205E31092830310567
:1006600010F0CD2B21F4DF91CF910C94BA06DF91DD
:10067000CF910C94C80681E0089581E008950C9410
:100680003D0308950C9441031F93CF93DF9300D053
:1006900000D00F92CDB7DEB749835A836B83309178
:1006A000AE0189819A8131111DC06623B9F02223E0
:1006B000A9F00E94B00A182F682F89819A810E94A0
:1006C000550A69817A81812F0F900F900F900F90BA
:1006D0000F90DF91CF911F910C94AF200E94840A5C
:1006E000182FEFCF0E94B00A69817A81EDCFFC010B
:1006F000262F86819781009739F44081518162814C
:10070000738184810C9444030895CF93DF93EC01AB
:1007100061E00E947703BE01DF91CF910C943127F5
:10072000CF93DF93EC0160E00E947703BE01DF917D
:10073000CF910C944203E1E0F0E0DF0102C0AA0F88
:10074000BB1F6A95E2F7BD01DF0102C0AA0FBB1F04
:100750004A95E2F76A2B01C0EE0F2A95EAF7962F29
:100760009823961302C08E2B0895E0958E2308954A
:10077000242F462F682F8091B4010E949B030C9474
:10078000120A0E94EA130E9428050C9405140E9484
:10079000082A0E94ED260E94C62A0C940814089587
:1007A0000E94E5060E94CF032FEF84E39CE02150D6
:1007B00080409040E1F700C000000C94BB2D0F93E7
:1007C0001F93CF93DF93EC018B010E946629B80140
:1007D000CE010E94B718882309F448C0B801CE01A1
:1007E0000E943F03882309F441C0B801CE010E9452
:1007F000AE298823D9F1B801CE010E94292B882384
:10080000A9F1B801CE010E94AB23882379F1B80188
:10081000CE010E94FD23882349F1B801CE010E9438
:100820002025882319F1F8018281882361F0CA35D7
:10083000FDE5DF0721F170F4C115ECE5DE07A1F05D
:10084000CE3DDC45C9F0C801DF91CF911F910F91DA
:100850000C943B03CB358DE5D807A1F0CC35DD45B5
:1008600091F70E94520FEFCF0E94D00380E0DF91FA
:10087000CF911F910F9108950E94FA10F7CF0E9417
:100880005B0FE1CF0E945E0FDECFCF93DF93EC01D1
:1008900061E00E947703BE01DF91CF910C94DF03EA
:1008A000DF92EF92FF920F931F93CF93DF93E82F86
:1008B000F0E0E451FF4FD490282F269526952695F9
:1008C00030E0F901E457FE4F0491877010E0082EE4
:1008D00002C0159507950A94E2F701701127F901F6
:1008E000E458FE4FE490F12C082E02C0F594E794F2
:1008F0000A94E2F791E0E922FF24F901E459FE4F5E
:10090000C491D0E002C0D595C7958A95E2F7C17031
:10091000DD270115110519F081EE0E94A805E114EB
:10092000F10419F086EE0E94A8058D2D0E94A706FD
:10093000EF2819F086EE0E943A06012B19F081EE9D
:100940000E943A06CD2B51F08CE2DF91CF911F919E
:100950000F91FF90EF90DF900C94A706DF91CF915D
:100960001F910F91FF90EF90DF900895EF92FF920B
:100970000F931F93CF93DF93EC01162F0AE088812A
:10098000882309F454C0813009F04EC08981813038
:1009900099F47E0122E0E20EF11C8A810E94A706F2
:1009A000E7012196812F815050F3EFE9FFE0319765
:1009B000F1F700C00000F7CF823041F47E0182E001
:1009C000E80EF11C8A810E94A805EACF833041F429
:1009D0007E01E2E0EE0EF11C8A810E943A06E0CF31
:1009E000843011F02196DDCF2A81229690E080E0BC
:1009F000AE014F5F5F4F2053330B2A30310548F073
:100A0000019778F2EFE9FFE03197F1F700C00000BD
:100A1000F7CF089FB001099F700D1124C901860FFF
:100A2000971F2981EA01E4CF0E945004BACFDF91D9
:100A3000CF911F910F91FF90EF90089560E00C947B
:100A4000B60408950C94210581E008950C942405C2
:100A50000895CF93C82F0E9422058C2FCF910C941C
:100A60002605019708F40895EFE9FFE03197F1F7C3
:100A700000C00000F6CFCF93DF93CDB7DEB72D9740
:100A80000FB6F894DEBF0FBECDBF49875A876B877C
:100A90007C878D878C859D85892B29F0CA018923C8
:100AA0008F3F09F046C08B8581110E94840F1D8203
:100AB0001E821F82188685E0FE013996DE0111969E
:100AC00001900D928A95E1F780914F049091500426
:100AD000892B61F00E941F0F882319F082E00E9489
:100AE00034100E94FB0E81110E94BE0F8C819D81EB
:100AF000892B99F429813A814B815C816D817E81BA
:100B00008F8198850E94440E2D960FB6F894DEBF13
:100B10000FBECDBFDF91CF91089589819A8189233E
:100B20008F3F41F3CE0101960E9485038111E2CFF0
:100B3000EBCF8091AF019091B00101969093B001FD
:100B40008093AF01B0CFFC01808191810C94DD0ACC
:100B5000CF93C82F882309F48BC08238C1F40E9438
:100B6000D02B81FD85C089E30E94E40E0E94CC0F4A
:100B70002FEF81EE94E0215080409040E1F700C0DB
:100B8000000089E30E94EB0ECF910C94CC0F8338C8
:100B9000A1F40E94D02B80FD6BC083E50E94E40E7F
:100BA0000E94CC0F2FEF81EE94E0215080409040C6
:100BB000E1F700C0000083E5E5CF8438A1F40E948E
:100BC000D02B82FD55C087E40E94E40E0E94CC0F1A
:100BD0002FEF81EE94E0215080409040E1F700C07B
:100BE000000087E4CFCF8CEF8C0F813A90F46C2F0C
:100BF00080910001909101010E94442C882329F0EA
:100C00008C2F0E94EB0E0E94CC0F8C2F0E94E40EC2
:100C1000BBCF80E28C0F883048F4C77081E001C000
:100C2000880FCA95EAF70E94640FAECFEBE5EC0F90
:100C3000E33040F4F0E0EE5AFE4F808190E0CF9137
:100C40000C94042CE8E5EC0FE73150F4F0E0EE0FE3
:100C5000FF1FEC5DFE4F80819181CF910C941A2C87
:100C6000C03F30F08C2F0E94E315CF910C94CE162C
:100C7000CF910895882309F452C0823871F40E94FC
:100C8000D02B81FF4CC089E30E94E40E0E94CC0F60
:100C900089E30E94EB0E0C94CC0F833859F40E9428
:100CA000D02B80FF3CC083E50E94E40E0E94CC0F55
:100CB00083E5EFCF843859F40E94D02B82FF2FC0F8
:100CC00087E40E94E40E0E94CC0F87E4E2CF9CEF01
:100CD000980F913AF0F290E2980F983050F48770A4
:100CE00091E001C0990F8A95EAF7892F0E946A0F57
:100CF000D2CF9BE5980F933020F490E080E00C94E5
:100D0000042C98E5980F973120F490E080E00C9443
:100D10001A2C803F20F00E944B160C94CE1608959A
:100D20001F93CF93DF93182FEB010E94A805209704
:100D300031F4812FDF91CF911F910C943A068FE906
:100D40009FE00197F1F700C000002197F0CF60917C
:100D50006D0470916E04893321F060916B04709181
:100D60006C040C949006882321F00E94640F0C946C
:100D7000CC0F0895882321F00E946A0F0C94CC0FA9
:100D80000895882321F00E94770F0C94CC0F0895CA
:100D9000882321F00E947D0F0C94CC0F089590E0E1
:100DA00080E00E94042C90E080E00E941A2C0E94B7
:100DB000840F0E94870F0E94CC0F0E94F5170C949D
:100DC000CE160E94F20E0C94CF060E94710F0C9466
:100DD000E106E92FE295EF70E250EE3070F4F0E0BA
:100DE000E05FF94C0C948135803F19F020F4883E87
:100DF00020F481E00895843FE1F380E00895883E87
:100E0000C0F3813FD1F7F5CF93FB882780F9089590
:100E1000FC0186819781009721F00E94FA110C94C1
:100E2000E906808191810E94DD0AF9CFBF92CF92BD
:100E3000DF92EF92FF920F931F93CF93DF937C018A
:100E4000EB01FC010281158112951F700E94390F80
:100E5000C82E8823A1F0C02E002389F08D2F807F1B
:100E6000803429F080E28C0FC12C883040F082E081
:100E70000E9434100E94390F91E0C82EC926BD2E61
:100E8000B2942FE0B222FBE0FB15B0F1EB2DF0E0C5
:100E9000E25EF94C0C9481352D2F2F70D22E8D2FC0
:100EA000807F19F0D29490EFD9220023A9F0DD20A1
:100EB00059F080E28C0F883010F0C11109C08D2DDF
:100EC0000E94640F0E94CC0F8C2F0E94A80514C0B2
:100ED0008D2D0E94770FF6CF8C2F0E943A06DD20D1
:100EE00059F080E28C0F883010F0C11134C08D2D84
:100EF0000E946A0F0E94CC0FEB2DE850FF0B349735
:100F000020F40E94D02B0E942905CE010E94E90600
:100F10008111D6C11092B0011092AF01CC2009F41A
:100F2000F0C10E941B0F80FDECC1F70112820E94EC
:100F3000150F0E94230AC7010E94A9090E94150FDC
:100F4000DF91CF911F910F91FF90EF90DF90CF90A5
:100F5000BF900C942E0A8D2D0E947D0FCBCF3D2F7C
:100F60003F70D32E8D2F807F803219F0D29480EF86
:100F7000D822CC23E9F0C13009F455C0002309F48C
:100F80005CC0112391F120E0F70140815181628121
:100F9000738184810E944403B7010E940A23811156
:100FA00093CFF701858180FF8FCF8F7085831DC020
:100FB0000023E9F0111106C00E948A0F8D290E94BA
:100FC000B3069ACF113031F40E948A0F8D290E9406
:100FD000A60F92CF80916904823070F38113ECCF19
:100FE0000E94BE0F8D2D0E94900F8D2DE8CF111104
:100FF00006C00E94BE0F8D2D0E94BA067DCF809143
:101000006904113059F4823008F476CF0E94610FE0
:101010008D2109F471CF0E94990FEBCF823048F3F4
:101020001813E7CF69CF002321F0163008F064CF02
:10103000DCCF153008F060CFDECF1123E1F28091D4
:101040006D0490916E04C93321F080916B049091EE
:101050006C040E9431058C2F0E943A064DCF8D2FD3
:1010600086958695837061F0813009F045CFCE0179
:101070009370011102C090E080E00E941A2C3CCFD6
:10108000CE019370011102C090E080E00E94042C18
:1010900033CF8C2F002339F00E94E3150E94CE1627
:1010A0000E94CE1629CF0E944B16FACF8D2F837047
:1010B00081F5011121CF4C2F429546954770440F81
:1010C000440F8C2F8F70042E01C0880F0A94EAF70A
:1010D0002C2F2071C4FF07C02FE030E001C0220F89
:1010E0004A95EAF720959D2F969596959370822BB9
:1010F000923049F058F4913019F00E94040AFCCE65
:101100000E94FF09F9CE0E94090AF6CE0E94FD094D
:10111000F3CE8695002311F08D2F8170882309F47A
:10112000EBCE4C2F429546954770440F440F8C2FC1
:101130008F70042E01C0880F0A94EAF72C2F2071BB
:10114000C4FF07C02FE030E001C0220F4A95EAF744
:1011500020959D2F969596959370822B923049F00D
:1011600058F4913019F00E944A0AC6CE0E94450AEE
:10117000C3CE0E944F0AC0CE0E94120ABDCEFD2FE0
:10118000FF70DF2E002329F08F2F0E94230A8C2F5F
:1011900016CF8C2F0E94BA068D2D0E942E0AACCE3F
:1011A000C23F09F43FC060F4C03F31F1C13F91F14B
:1011B000002309F480C0111187CE8D2F8F712FC0AD
:1011C000C33FA9F1C43FA1F780916904823008F4BC
:1011D0005BC0002309F444C00E94F80E0E946A0F0D
:1011E0000E941B0F843069F50E942B108D2F8F7188
:1011F0000E942E0AC12C80CE002341F0153008F049
:101200007BCE8D2F8F710E943A0A76CE163008F071
:1012100073CEF7CF8D2F8F71002309F4BECF0E94BC
:10122000230A6ACE8D2F8F710023C9F3B6CF002316
:1012300029F08D2F8F710E941B0A5ECE0E94180A22
:101240005BCE809169041817A8F62D2F2F71D22E2E
:10125000822F0E94230A63E08D2D0E940F10CACFB7
:101260000E94F80E0E94640F80916904181740F0E4
:101270000E942B100E94990F64E08D2F8F71EDCF8B
:1012800081E00E943410B6CF002359F03D2F3F710A
:10129000D32E832F0E94230A63E08D2D0E940F100E
:1012A0002BCE81E00E943410123008F425CE82E06B
:1012B0000E94341021CE1111C2CE8D2F8F716DCFAF
:1012C000002319F0111126CE29CE111123CE20E0D2
:1012D000F701408151816281738184810E944403BE
:1012E000B7010E941523882309F414CE8091AF0121
:1012F0009091B001029709F00DCE8C2F0E94A706A5
:1013000009CEDF91CF911F910F91FF90EF90DF9069
:10131000CF90BF9008950F931F93CF93DF93EC016D
:101320008E819F81009779F00E94FA118C010E94B2
:10133000540A0E94FC09B801CE01DF91CF911F91A0
:101340000F910C941607688179818A810E94E70ABF
:10135000EDCFCF93DF93EC018B819C81892B29F01A
:101360008881998189238F3F59F4DF91CF91089526
:10137000CE010E948B09CE01DF91CF910C94900396
:10138000CE010E9445048111F3CF0E94390F8823BA
:1013900061F38A81882349F382E0DF91CF910C9435
:1013A0003410CF93DF9300D000D00F92CDB7DEB7CB
:1013B0000F900F900F900F900F90DF91CF910895A5
:1013C000CF93DF93CDB7DEB728970FB6F894DEBF83
:1013D0000FBECDBF28960FB6F894DEBF0FBECDBFAF
:1013E000DF91CF91089508950C94F3090E94F409B8
:1013F0008093B5010C94CF0608950C94F609909152
:10140000B501892B0C94F6099091B50189230C94B0
:10141000F6099091B50189270C94F6090C94F3090B
:101420000C940E0A0E94100A8093B4010C94CF060B
:1014300080E00C94120A91E001C0990F8A95EAF7B6
:10144000892F0C94120A21E030E001C0220F8A9506
:10145000EAF78091B401822B0C94120A21E030E06B
:1014600001C0220F8A95EAF720958091B40182236A
:101470000C94120A21E030E001C0220F8A95EAF7AD
:101480008091B40182270C94120A9091B401892BA7
:101490000C94120A9091B40189230C94120A909131
:1014A000B40189270C94120A08959E3F61F1990FA7
:1014B000990FE92FE80F8E2F877041E001C0440F8C
:1014C0008A95EAF7E695E695E69583E0E89FF001D0
:1014D0001124EF54FE4F30E020E070E05191DF0125
:1014E0001197CB01022E02C0969587950A94E2F7D8
:1014F000817081958527842385278C932F5F3F4FAB
:101500002330310559F708959E3F41F1990F990F06
:10151000E92FE80F9E2F9770E695E695E69583E014
:10152000E89FF0011124EF54FE4F50E040E080E0CE
:10153000219130E0092E02C0369527950A94E2F7F2
:1015400021703327042E01C0220F0A94EAF7822B60
:101550004F5F5F4F4330510559F7089580E008957C
:10156000CF92DF92FF920F931F93CF93DF936C0183
:101570000091B4018091B501082BC7E0D0E010E0E4
:10158000FC2EC8010C2E02C0959587950A94E2F7AF
:1015900080FD0CC02197A0F7F12C8F2DDF91CF910A
:1015A0001F910F91FF90DF90CF900895B6018C2F7F
:1015B0000E94F212019771F3F0CFCF93DF93EC0109
:1015C0000E94B00ABE01DF91CF910C94F2121F93DA
:1015D000CF93DF93EB019091AE01992331F0CB01D2
:1015E000DF91CF911F910C94DD0A882379F0CB0114
:1015F0000E94B00A182F682FCE010E94550ABE0122
:10160000812FDF91CF911F910C94F212CB010E9498
:10161000840A182FF4CFCF93DF93C091B601809145
:10162000B7018C1303C0DF91CF910895D0E0FE0184
:1016300083E0EE0FFF1F8A95E1F7E854FE4F20810B
:1016400031814281538164817581868197810E94B5
:10165000E0092196C770E3CF2091F8013091F9019C
:101660004091FA015091FB016091FC017091FD01E4
:101670008091FE019091FF010C94E0092091B60148
:101680009091B701291302C080E0089530E0F9017C
:1016900053E0EE0FFF1F5A95E1F7E854FE4F5181DA
:1016A000561306C05081581303C05281541304C00E
:1016B0002F5F3F4F2770E6CF81E00895EF92FF92B2
:1016C0000F931F93CF93DF938091FD01807F31F4BF
:1016D0008091FA01C091B601811119C0DF91CF91BB
:1016E0001F910F91FF90EF9008952091FB01309191
:1016F000FC01D0E02115310541F08091F801909175
:10170000F901482F49234F3F39F42196C770809142
:10171000B7018C13EACFE2CF8E0143E0000F111F17
:101720004A95E1F7F801E854FE4F41814913EDCFA6
:1017300090819813EACF82818111E7CFE380F48012
:10174000E21AF30A60E088EF91E00E94770368EF05
:1017500071E00E940123E816F906B8F68091FD01B8
:101760008F7080618093FD01F801E354FE4F80810A
:101770008F708061808388EF91E00E94A909DF91DA
:10178000CF911F910F91FF90EF900C940B0B6F92E4
:101790007F928F929F92AF92BF92CF92DF92EF9201
:1017A000FF920F931F93CF93DF93CDB7DEB765976B
:1017B0000FB6F894DEBF0FBECDBF8C0185E0F801F7
:1017C000DE01519601900D928A95E1F7D8011296AB
:1017D000FC90129788EF882E81E0982E2091FB01D3
:1017E0003091FC012115310541F08091F801909173
:1017F000F90189238F3F09F0E9C1F11010C1C80137
:101800000E94A90982C060E088EF91E00E947703FE
:10181000B8010E940623811116C2CD2829F0872D18
:1018200086218F3F09F011C180E0B82FB170CB2E17
:1018300080FF29C04F2D672D862D0E943E0BD82E8C
:10184000811121C0698A7A8A89899A890E94DD0A70
:10185000292F22952F70223050F0243078F49F7079
:1018600051F0F8019581907F31F4ED2C1AC19F70F1
:1018700011F08823D1F3805E8830B8F3C8010E944C
:10188000A909DC2CF2CFFF2009F40BC18091FD01E6
:1018900081608093FD01E12C04C1892B49F0809186
:1018A000F8019091F901282F29232F3F09F00FC14A
:1018B000C8010E940807882309F4A1CFFF2009F47A
:1018C0009ECF8091FD018032A0F02091F8013091EF
:1018D000F9013A8729871B86DD86CC868E87809121
:1018E000FE019091FF01988B8F87CE0109960E948F
:1018F000A90988E0F801A8EFB1E001900D928A955E
:10190000E1F70E945E0B0E942C0BEE24E394C9C009
:10191000211112C07C2DDD8ACC8AA3016F2D8D8907
:101920000E94D10988EF91E00E94A90988E0F401A2
:1019300011928A95E9F7A5C18091FB019091FC0174
:10194000892B49F08091F8019091F901282F2923E2
:101950002F3F09F0E4C0C8010E940807882309F45A
:101960004ECFFF2009F44BCF8091FD01803208F269
:101970002091F8013091F9013A8329831B82DD829D
:10198000CC828E838091FE019091FF0198878F8396
:10199000CE010196ACCF60E088EF91E00E94770322
:1019A00068EF71E00E940123A816B90650F5EF2CEC
:1019B000FF2009F424CF8091FB019091FC01892B39
:1019C00049F08091F8019091F901282F29232F3FA8
:1019D00009F0CBC0C8010E94080781118ACF80910D
:1019E000FD0181608093FD01C8010E94A90959C0D1
:1019F00088E0F801A8EFB1E001900D928A95E1F737
:101A000050C07C2DDD8ACC8AA3016F2D8D890E9468
:101A1000D10988E0F40111928A95E9F77DC0C801E7
:101A20000E940807E82E882309F4E9CE88E0F8012F
:101A3000A8EFB1E001900D928A95E1F788EF91E06F
:101A40000E94A3050E945E0B67C081E08F25EDCE4A
:101A500081E08F2501C1D80111962C912913E7C08F
:101A6000F80190819813E3C02091FE013091FF01AD
:101A7000868197812817390709F0D9C0F110D7C09E
:101A80008091FD018F7080618093FD010E942C0B7D
:101A900088EF91E00E94A9098091FD01D801159677
:101AA0008C938E2D65960FB6F894DEBF0FBECDBF1A
:101AB000DF91CF911F910F91FF90EF90DF90CF902A
:101AC000BF90AF909F908F907F906F900895F80196
:101AD00021812913EDCED8019C919813E9CE209154
:101AE000FE013091FF0116968D919C911797281752
:101AF000390709F0DDCE8091FD01F110D9CE1596A0
:101B00008C93C8010E94A90988E0F801A8EFB1E010
:101B100001900D928A95E1F70E942C0BC2CFD8015B
:101B200011962C91291317CFD8019C91981313CF9C
:101B30002091FE013091FF0116968D919C9117978F
:101B40002817390709F007CFF11005CF8091FD0163
:101B500015968C93C8010E94A909E8EFF1E088E08E
:101B6000DF011D928A95E9F79CCFF80121812913A5
:101B700031CFF801908198132DCF2091FE01309143
:101B8000FF01868197812817390709F023CF60E08C
:101B900088EF91E00E947703B8010E940F23811122
:101BA00027CF8091FD0180FD23CF982F907F09F4EE
:101BB0001FCFD80115968C931597903F09F4A1CFAC
:101BC000982F907F905F8F70892B99CF6C90119692
:101BD0007C9011971396CD90DC90E090FA0156011D
:101BE000A21AB30AEE2009F4D6CE60E088EF91E0A5
:101BF0000E94770368EF71E00E9401232091FD01AC
:101C0000207FA816B90608F083CE8091FB01909141
:101C1000FC01211142CEEF2C892B49F08091F80173
:101C20009091F901282F29232F3F09F014CF60E06C
:101C300088EF91E00E947703B8010E940123843F5E
:101C4000914008F4E0CDC114D10429F0872D8621FC
:101C50008F3F09F0FDCE80E080FFDFCD4F2D672D57
:101C6000862D0E943E0B882309F4D7CD88EF91E0A2
:101C70000E94A90988E0E8EFF1E0DF011D928A9552
:101C8000E9F70E942C0B07CECF93DF93CDB7DEB7D9
:101C900060970FB6F894DEBF0FBECDBF29873A8795
:101CA0004B875C876D877E878F87988BCE010996DF
:101CB0000E94C70B8823D1F08C859D85892B39F034
:101CC00029853A85822F83238F3F09F074C0809144
:101CD000B6019091B701891348C060960FB6F89489
:101CE000DEBF0FBECDBFDF91CF91089588E0FE012A
:101CF0003996DE01119601900D928A95E1F78C8557
:101D00009D85892B21F389859A8589238F3FF9F257
:101D1000A091B701B0E0CD0101968770992720917D
:101D2000B6012817190671F40E94E5061092B70152
:101D30001092B60188E0E8EFF1E0DF011D928A958C
:101D4000E9F7C5CF93E0AA0FBB1F9A95E1F7A85416
:101D5000BE4F98E0FE01319601900D929A95E1F701
:101D60008093B7010E940B0BB2CFB8E08B9FC001EC
:101D7000112488549E4F0E94C70B882309F4ADCFCD
:101D8000E091B60128E0E29FF0011124E854FE4FF3
:101D9000208131814281538164817581868197815F
:101DA0000E94E0098091B60190E001968770992722
:101DB0008093B6018CCF4B855C856D857E858F8544
:101DC00098890E94E00983CF682F8091000190914B
:101DD00001010C94C42C682F8091000190910101A5
:101DE0000C94CF2C80910001909101010C94DA2C7D
:101DF00080910502089580914F0490915004892BA1
:101E000089F00E94702D2091030230910402AC01F0
:101E1000421B530B81E020914F0430915004421734
:101E2000530708F480E0817008958091020285953F
:101E300085958595089580910202877008950E9486
:101E4000702D2091000230910102821B930B209192
:101E50004F04309150048217930748F0809102029A
:101E600082FB882780F991E089278170089580E0BE
:101E7000FCCF90910202977081E009F480E0089510
:101E80009091F60392FB222720F9281751F080FB4E
:101E900092F99093F6038091F5039091F6030C94D8
:101EA000771008958091F60382FB882780F991E0EE
:101EB00089270C94400F81E00C94400F80E00C9433
:101EC000400F80912902089590912902892B8093D7
:101ED00029020895809590912902982390932902D0
:101EE00008951092290208958091280208959091F2
:101EF0002802892B809328020895809590912802CA
:101F00009823909328020895109228020895109221
:101F10002702089580910602089508950C948D0F6C
:101F200090910502981721F0809305020C948E0F72
:101F3000089580910502882329F01092050280E01F
:101F40000C948E0F089508950C94A30FCF93C82F6F
:101F50008091F60382FD10C0809106028C1761F01B
:101F60000E94702D9093040280930302C093060296
:101F70008C2FCF910C94A40FCF91089580910602DD
:101F8000882349F010920602109204021092030274
:101F900080E00C94A40F0895E0910001F0910101FC
:101FA000809129028083E0910001F09101018081FC
:101FB00090912802892B8083E0910001F09101012A
:101FC000808190912702892B80838091060288234B
:101FD000E9F080914F0490915004892B29F00E94E0
:101FE000FB0E81110E94BE0FE0910001F0910101F2
:101FF000808190910602892B8083809100019091CD
:1020000001010E94302C81110E94BE0F80910001BD
:10201000909101010C94DC2B08950C940C1090917C
:10202000F60392FD16C098E0899F90011124622B5F
:10203000609302020E94230A0E94702D9093010275
:1020400080930002809102028595859585950C9478
:102050000D100C94230A10920202109201021092A9
:10206000000280E00C940D1090910202809589236B
:1020700080930202282F277039F4282F082E000C95
:10208000330B9217130621F49091F60392FF07C0C9
:102090008595859585950E942E0A0C942B100895A0
:1020A0006FEF7FEF90E080E00C94F03590E080E0FF
:1020B0000E94CC358A3E9E4F11F40C94601880E04B
:1020C000089582E090E00C94C43583E090E00C9495
:1020D000C435CF9384E090E00E94C435C82F82E2DB
:1020E00090E00E94C435982F8C2FCF910895CF9304
:1020F000C92F682F84E090E00E94D2356C2F82E2D5
:1021000090E0CF910C94D235AB01BC018FE090E010
:102110000C94E435AB01BC0183E190E00C94E43510
:1021200060E070E0CB010C948A1060E070E0CB01BD
:102130000E9484100C9490106AEE7EEF90E080E094
:102140000E94F03560E082E090E00E94D23560E0CD
:1021500083E090E00E94D2351092B50160E084E007
:1021600090E00E94D23560E082E290E00E94D23599
:1021700060E085E090E00E94D23560E086E090E08B
:102180000E94D2356FEF87E090E00E94D23540E0A8
:1021900050E0BA0188E090E00E94E43560E08DE014
:1021A00090E00E94D23540E050E0BA0188E190E032
:1021B0000E94E43560E087E190E00E94D23540E083
:1021C00050E0BA018CE190E00E94E43570E060E0FC
:1021D00080E290E00E94F03540E050E0BA0188E1F2
:1021E00090E00E94E43580E00E9479180E949F18D8
:1021F0000C9495100C949C10682F8EE090E00C9439
:10220000D2350E947C2D6093350270933602809304
:1022100037029093380260933102709332028093B8
:1022200033029093340208950E947C2D609335020E
:1022300070933602809337029093380260932D0298
:1022400070932E0280932F0290933002089585B7E9
:10225000806885BF85B7806885BF08950895089513
:102260000C942E1108950C9432110E94271180EDC8
:1022700093E10E94DF2D0E942D1C0E940F220E94DC
:102280002F110C94301181E008950C94431108959E
:1022900008950E9447110C9448110E94672D0E94D6
:1022A000AE180E94C1140E9403180C943311AF920F
:1022B000BF92CF92DF92EF92FF920F931F93CF9333
:1022C000DF93CDB7DEB72A970FB6F894DEBF0FBE07
:1022D000CDBF0E94D11481110E9401118BE2A82E62
:1022E00082E0B82E10E000E0C02E802F0E941E1465
:1022F000E82EF501F1905F01F81609F456C08091BF
:10230000390281FD0E9424148F2D8E25D12CFF24AB
:10231000F394982F9F2109F443C00E94451188230C
:1023200099F0DE82CF82EF2081E009F480E0888797
:102330000E94702D8160782F9A8789874E815F81F6
:1023400068858A850E943B05F801E55DFD4F808127
:10235000F826F0820E94161881110E9414110E9422
:10236000E9160E94D02B90912A02891791F10E94C0
:10237000D02B80932A022A960FB6F894DEBF0FBEA8
:10238000CDBFDF91CF911F910F91FF90EF90DF9024
:10239000CF90BF90AF900C94290501E010E0A4CF3E
:1023A000D394FF0CF4E0DF12B4CF01301105A9F78C
:1023B0008FEF89838A831B820E94702D8160782F22
:1023C0009D838C8349815A816B818D810E943B055D
:1023D000C1CF2A960FB6F894DEBF0FBECDBFDF91F6
:1023E000CF911F910F91FF90EF90DF90CF90BF9012
:1023F000AF900895CF93DF930E94F612EC01811500
:1024000021E5920708F042C0811530E5930708F0F6
:102410009DC0883E910530F5803E910508F092C040
:10242000883A910588F4853A910508F084C0813096
:10243000910509F487C0009709F484C0049708F057
:1024400081C0D0E0C0E07EC08F3B9105D0F7C85A74
:10245000D0E0CC0FDD1FCB5ADE4F0990D881C02DC4
:10246000D46470C08115904250F4C11581E0D80742
:1024700008F068C0C03FD10520F3D06563C0C11526
:1024800090E4D907F0F2DF70D06A5CC0811525E5D1
:10249000920700F5811534E5930708F08BC081158C
:1024A00043E5940708F073C0C11582E5D80708F426
:1024B00069C0CE018370992721E030E002C0220F6D
:1024C000331F8A95E2F7C695C69580E2C89FE00162
:1024D000112454C0C11599E5D907A8F4C11528E500
:1024E000D20708F06CC0C11536E5D30708F0A9CFB4
:1024F0008C2F0E948D13C82FD0E0DC2FCC27CC2747
:10250000DF71D0621FC0C1154AE5D40708F45CC072
:10251000CE0190568115904208F093CF8D2F8F7188
:102520000E948D1390E0982F882788279F719C0127
:102530002C2BE901E6CFC55AD0E0CD57DE4FC8813C
:10254000D0E0D064CE01DF91CF910895E4E096957C
:102550008795EA95E1F783702C2F269526952370B1
:1025600040E2249F90011124382B8C2F8370C1E00E
:10257000D0E002C0CC0FDD1F8A95E2F7C22BD32B2F
:10258000DC68E0CFDC2FCC27C16FD06ADBCF837053
:10259000992721E030E002C0220F331F8A95E2F72D
:1025A000C695C69590E2C99FE0011124C22BD32B9A
:1025B000DA68C8CFD82FCC27C46FD06AC3CFDC2F3E
:1025C000CC27C06FD06ABECF8C2F8F700E948D1326
:1025D00034E0D695C7953A95E1F7CF709C2FEC0182
:1025E000D069B0CF0E94AF200C94FA1182389105C7
:1025F000B1F1B0F48133910509F475C048F4893222
:10260000910509F469C08A32910509F473C00895EF
:102610008533910509F459C08933910501F1089575
:10262000833E9105A9F138F4803E9105F9F0823E90
:10263000910549F10895863E9105A9F1873E9105DE
:10264000C9F1843E910519F52091F60321FF1FC0C1
:102650008091F50384FD14C087EE90E008952091E9
:10266000F5032370A1F080EE90E008952091F5032A
:1026700020FD47C03091F60330FF09C024FF44C05D
:1026800090E080E004C02091F50322FDF7CF08958B
:102690002091F50322FD3BC03091F60330FDE3CFDE
:1026A00024FFF5CFEDCF2091F50323FFF0CF24FDDC
:1026B000E7CFD2CF2091F50323FD2CC03091F60354
:1026C00031FFEECF84EE90E008952091F50325FFD1
:1026D000DECF89E290E008952091F50325FFD7CF62
:1026E00085E390E008952091F50326FFD0CF8AE29C
:1026F00090E008952091F50326FFC9CF81E390E093
:10270000089589E390E0089583EE90E0089582EEC5
:1027100090E0089586EE90E008959091F50392FF81
:1027200006C0282F28712830F9F4877F846093FF32
:1027300006C0282F28712831F1F4877E846120910A
:10274000F60320FF06C0382F38713830D9F4877F60
:10275000816021FF06C0282F28712831D1F4877E9F
:10276000816194FD877E0895282F24712430F9F625
:102770008B7F8860DCCF282F2471243101F78B7E7A
:102780008861DDCF382F3171313019F78E7F886045
:10279000E0CF282F2171213121F78E7E8861E1CF92
:1027A00080E008950C9450100E94D1148FE39CE9AE
:1027B0000197F1F700C000000E94D11480E00E9450
:1027C0001E1480FF04C00E94D2130C94BB2D0895E8
:1027D0000C94D4130E945610811102C00E94FA106A
:1027E0000E946110809339020E9469109093F60351
:1027F0008093F5030E94E8130E9465100E94FD0972
:102800008091B4010C94100A08950C940414089556
:102810000C940714E82FF0E0E750FC4F208130E0E3
:1028200081E090E002C0880F991F6A95E2F72823A3
:10283000392381E0232B09F480E00895E82FF0E0AC
:10284000E750FC4F80810895089580EA8A95F1F75A
:10285000089500C008950C942514F894E82FE2958B
:10286000EF70F0E031A1282F2F7081E090E001C0DF
:10287000880F2A95EAF7982F9095932391A392A118
:10288000892B82A37894089585E30E942D1484E314
:102890000E942D1486E30E942D1486E60E942D14BA
:1028A00087E60E942D1484E90C942D14CF92DF92B8
:1028B000EF92FF920F931F93CF93DF93EC01D62EED
:1028C000062F10E0C80186579E4F7C01FC018081D5
:1028D0008F3F09F44BC0F894E82FE295EF70F0E0D9
:1028E00091A18F7021E030E001C0220F8A95EAF7B4
:1028F000892F822B81A382A12095282322A378945B
:102900000E942914E6E8F1E030E020E0C12C51E01B
:1029100041914F3FA1F1A42FA295AF70B0E09096E6
:102920008C9190E04F7002C0959587954A95E2F79B
:1029300080FD25C0852F022E01C0880F0A94EAF77A
:10294000C82A2F5F3F4F2430310511F7F7018081EE
:102950008F3F11F00E942D1461E0C11001C060E0B2
:102960008D2D0E942B14C00FD11FC882DF91CF91F3
:102970001F910F91FF90EF90DF90CF90089580E02E
:10298000DFCF0E944414A7EFB3E01C92E9EFF3E01D
:10299000108211961C92118282E00E9409150C94FB
:1029A000C1031F93CF93DF9300D0CDB7DEB71A8258
:1029B000198260E0CE0101960E94561461E0CE01BA
:1029C00001960E94561442E050E0BE016F5F7F4FB7
:1029D00087EF93E00E94973511E0009709F410E02B
:1029E000892B31F089819A819093F8038093F703C2
:1029F000212F42E069EF73E087EF93E00E940A1510
:102A00000E94C703812F0F900F90DF91CF911F91EC
:102A100008950895FF920F931F93CF93DF93F82E9D
:102A2000092F162FD72FC42F222349F081E080933E
:102A30003C020E94702D90933B0280933A02809159
:102A40003C028823A1F080913A0290913B020E94BF
:102A5000882D059760F0EF2DF02FA12FBD2FCE0F01
:102A6000DF2FD11DEC17FD0741F410923C02DF91DE
:102A7000CF911F910F91FF90089581918D93F2CF87
:102A80000E94EC2C0E94852F0E949E2F0E94B02F46
:102A90000E944911FBCF80914302609155047091CF
:102AA000560480FF16C020910701269FC001279F72
:102AB000900D1124BC0176956795769567956038E1
:102AC000710508F043C06115710509F441C0862FF6
:102AD000089581FF0BC020910701269FC001279F09
:102AE000900D1124BC0176956795E9CF82FF09C04E
:102AF000809107019B01829FB001839F700D11247B
:102B0000DECF209142022223D1F2909106018091E2
:102B10000701482F50E0291748F0CB01849FB001EE
:102B2000859F700D949F700D1124C9CF289F90012F
:102B30001124269FA001279F500D369F500D112470
:102B4000692F70E0CA010E945935B9CF8FE7089507
:102B500081E008958091430280FF0CC060910301E1
:102B600070E075956795759567956115710549F1E3
:102B7000862F089581FF06C06091030170E075956E
:102B80006795F3CF6091030182FD0BC090914102E4
:102B90009923A1F06091020180910301961738F00A
:102BA000682F70E06038710500F38FE70895899F02
:102BB000C001112470E00E946D35F4CF61E070E037
:102BC000D7CF81E00895803F31F40E944B15819565
:102BD000809347020895813F19F40E944B15F8CF66
:102BE000823F31F40E944B158195809346020895EF
:102BF000833F19F40E944B15F8CF893F29F40E94B6
:102C0000AA158093480208958A3F21F40E94AA15CC
:102C10008195F7CF8B3F31F40E94AA15819580935F
:102C2000490208958C3F19F40E94AA15F8CF843FF9
:102C300031F4809145028160809345020895853F7B
:102C400021F4809145028260F7CF863F21F4809184
:102C500045028460F1CF873F21F48091450288606E
:102C6000EBCF883F21F4809145028061E5CF8D3F15
:102C700031F48091430281608093430208958E3F36
:102C800021F4809143028260F7CF8F3FB9F78091A2
:102C900043028460F1CF90914602803F59F48091C5
:102CA000470287FF0DC01092470291110BC010928E
:102CB000420208C0813F81F48091470218169CF3BC
:102CC000992381F08091480290914902892B09F063
:102CD00064C0109241020895823F49F497FFF0CFFB
:102CE00010924602809147028111ECCFE0CF833FE2
:102CF00019F41916ACF3E4CF20914802893F29F466
:102D00001216F4F610924802DBCF8A3F19F427FF1F
:102D1000D7CFF8CF209149028B3F29F427FFD0CF9E
:102D200010924902CDCF8C3F19F41216CCF3C8CFC4
:102D3000843F31F4809145028E7F80934502C0CF5D
:102D4000853F21F4809145028D7FF7CF863F21F4A6
:102D5000809145028B7FF1CF873F21F4809145021E
:102D6000877FEBCF883F21F4809145028F7EE5CFAE
:102D70008D3F31F4809143028E7F80934302A0CF38
:102D80008E3F21F4809143028D7FF7CF8F3F09F072
:102D900097CF809143028B7FF0CF08950E94702DD2
:102DA0009C019091460280914702982B21F030932C
:102DB000400220933F029091480280914902982B53
:102DC00021F030933E0220933D0284E492E00C9483
:102DD000F62BEF92FF920F931F93CF93DF9300D0C8
:102DE00000D000D0CDB7DEB786E0E4E4F2E0DE014B
:102DF000119601900D928A95E1F7E0904602F090CD
:102E00004702009148021091490210924602109226
:102E1000470210924802109249028E2D8F2991F09C
:102E200080913F02909140020E94882DAC019091C8
:102E30004202992309F43FC08091080184171506C6
:102E400008F447C0802F812B91F080913D02909132
:102E50003E020E94882DAC0190914102992309F411
:102E600077C0809104018417150608F47FC0809113
:102E7000460290914702892B90914802892B9091AC
:102E80004902892B11F00E94CE1686E0FE01319690
:102E9000A4E4B2E001900D928A95E1F726960FB670
:102EA000F894DEBF0FBECDBFDF91CF911F910F9180
:102EB000FF90EF900895209109018AE0289F9001EA
:102EC00011242417350708F0BDCF9F5F909342026D
:102ED00002C09F3FD1F7EE2059F00E944B159FEFA3
:102EE0001E140CF491E0899F802D112480934602DA
:102EF000FF2059F00E944B159FEF1F140CF491E036
:102F0000899F802D112480934702309146023323FC
:102F100009F498CF20914702222309F493CF45EB7F
:102F20003403C0011124992359F09093460245EBD4
:102F3000240390011124332339F03093470282CFC8
:102F400081E080934602F3CF81E0809347027ACFFD
:102F5000209105018AE0289F90011124241735074C
:102F600008F085CF9F5F9093410202C09F3FD1F749
:102F7000002359F00E94AA159FEF10160CF491E05F
:102F8000899F802D112480934802112359F00E94BB
:102F9000AA159FEF11160CF491E0899F802D112442
:102FA0008093490230914802332309F460CF209185
:102FB0004902222309F45BCF45EB3403C0011124FD
:102FC000992359F09093480245EB24039001112472
:102FD000332339F0309349024ACF81E0809348028D
:102FE000F3CF81E08093490242CF86E0E4E4F2E04F
:102FF000DF011D928A95E9F7109242021092410278
:1030000010924302089557985F9A56985E9A89B134
:1030100090E0880F892F881F990B4E9905C020E0FA
:10302000822B80934C02089522E0FACFE0914C026B
:10303000EE0FEE0FE0934C0289B190E0880F892FDC
:10304000881F990B49B146FB222720F946FF02C091
:1030500022E030E0822BE82BE0934C02EF70F0E0AE
:10306000E457FE4F808190914B02890F80934B0271
:1030700020E0843054F080914A028F5F80934A02AE
:1030800060E080E00E94F41D21E080914B028D3FC2
:1030900054F480914A02815080934A0261E080E0BA
:1030A0000E94F41D21E080914B02082E000C990B28
:1030B00064E070E00E946D3580934B02822F08958A
:1030C00083E290E00E94C435823C89F484E290E07F
:1030D0000E94C435843959F485E290E00E94C435D9
:1030E00091E08A3209F090E0892F8170089580E0A4
:1030F000FCCFCF93C82F6FEF811162EC83E290E099
:103100000E94D2356FEFC11164E984E290E00E9421
:10311000D2356FEFC1116AE285E290E0CF910C9455
:10312000D235089586E290E00E94C435682F70E0A1
:1031300090E080E0089586E290E00C94D23580E043
:103140000E94791860E070E0CB010E949B180E94F9
:10315000561F0E94222181E00C9479180E94911838
:103160000E946018811102C00C949F180895CF939B
:10317000FB01C281CC2309F19C0122513F45203142
:10318000310520F582510E943221C0E08C2FCF9171
:10319000089581E00E94230A43E062E081E00E94FA
:1031A000B803F3CF81E00E942E0A43E062E081E0A1
:1031B0000E94B803EBCF82E0F6CF8031FFE59F0796
:1031C00089F381319F45B9F3C1E0E0CF8031EFE56C
:1031D0009E07F9F281319F45C9F682E0DBCF2FEFE0
:1031E000FC01208308951F93CF93DF93EC01162FEA
:1031F000888120914B0330914C03232B79F08E3F33
:1032000009F05CC08981833020F08550833008F05C
:1032100055C0612FCE010E94311C50C08B3009F483
:10322000E2C0D0F4843009F480C060F4823009F444
:103230004CC008F06DC08130F1F1612FCE010E94C9
:10324000EF183CC0863009F486C008F479C08A3093
:10325000A0F78FEF888332C0803109F49CC000F55D
:103260008D3009F47FC008F479C08E3009F482C033
:103270008F3019F780914D0390914E03892BF1F017
:103280006B8170E06D317105C8F489819A81AE015E
:103290004C5F5F4F9827892798270E94F7200EC020
:1032A000823109F47EC008F479C0833109F48AC000
:1032B0008E3F19F6AECF198289E08A83612FCE0145
:1032C000DF91CF911F910C947A2E8981823071F019
:1032D000833079F0813009F0B0CF0E947C2D0E94BC
:1032E00087356A837B838C839D83E8CF0E94921805
:1032F000F6CF80914D0390914E03892BF9F280E037
:103300000E941E148A8381E00E941E148B83D6CFF4
:103310008981823009F091CF6A817B818C819D8186
:103320000E9487350E949B18C9CF4B816A81898191
:103330000E944F1E9827892798279D838C83BECF94
:103340002C813D813227232732274B816A81898155
:103350000E94711EB3CF0E94561FB0CF0E94CB2097
:103360008983ACCF0E94CD209827892798279A83FC
:103370008983A4CF6B8170E06D31710508F09ECF19
:1033800089819A81AE014C5F5F4F982789279827E2
:103390000E94D02093CF0E94222190CF0E943C1EF9
:1033A000DFCF6B8170E06D31710508F087CF8981C7
:1033B0009A81AE014C5F5F4F9827892798270E941A
:1033C000F91F7CCF6B8170E06D31710508F076CF0D
:1033D00089819A81AE014C5F5F4F98278927982792
:1033E0000E941E206BCF80914D0390914E03892B3C
:1033F00009F464CFCE010E947A2E2FEF81EE94E083
:10340000215080409040E1F700C000000E94BB2D99
:1034100055CF8F929F92AF92BF92CF92DF92EF9251
:10342000FF920F931F93CF93DF93CDB7DEB72A9709
:103430000FB6F894DEBF0FBECDBF05E812E0F12C49
:10344000E12C87E8C82E8BE1D82E91EBA92E9BE1C9
:10345000B92E2EE8822E2AE1922EF801D182C08266
:10346000B382A28295828482F58AE48ABE016F5F6C
:103470007F4F8E2D0E94061F892B29F489859A85FE
:10348000F801938B828BFFEFEF1AFF0A0A5E1F4F42
:1034900088E0E816F10409F72A960FB6F894DEBF23
:1034A0000FBECDBFDF91CF911F910F91FF90EF9095
:1034B000DF90CF90BF90AF909F908F900895CF9363
:1034C000DF9300D000D00F92CDB7DEB790934C04BD
:1034D00080934B04811520E2920748F40F900F90DF
:1034E0000F900F900F90DF91CF910C9423038EEFEC
:1034F00089838A831B820E94702D8160782F9D832F
:103500008C8349815A816B818D810F900F900F9030
:103510000F900F90DF91CF910C943B050F931F9369
:10352000CF93DF938C01EB0165E373E08C2F0E9456
:10353000061F892BA1F480916B0490916C04019774
:1035400098F4DD27C15CDC4F8881F8011082188275
:10355000833041F180F4813091F08230B9F0DF9115
:10356000CF911F910F910895EFE9FFE03197F1F7A7
:1035700000C00000E4CF8430D1F0853081F7809125
:10358000350390913603009751F306C080913703BD
:1035900090913803009799F3DF91CF911F910F918C
:1035A0000C945F1A8091390390913A03F3CF809184
:1035B0003B0390913C03009779F7209135033091BC
:1035C0003603809137039091380321153105D9F2E4
:1035D000009711F7C901E0CFCF93DF9300D000D05F
:1035E0000F92CDB7DEB790934C0480934B048115B6
:1035F00020E2920748F40F900F900F900F900F90D9
:10360000DF91CF910C940C038EEF89838A8381E044
:103610008B830E94702D8160782F9D838C834981DC
:103620005A816B818D810F900F900F900F900F90AA
:10363000DF91CF910C943B05CF92DF92EF92FF92F6
:103640001F93CF93DF93CDB7DEB72A970FB6F894C9
:10365000DEBF0FBECDBFEBEFF3E080E5DF011D92D3
:103660008A95E9F7EDE4F2E088E3DF011D928A959F
:10367000E9F78BEFC82E83E0D82E7F0110E0F70129
:10368000D182C082BE016F5F7F4F812F0E942E1FAB
:10369000892B79F488E0FE013196D60101900D92D4
:1036A0008A95E1F789859A85D70113969C938E9325
:1036B0001297BAE0CB0ED11CE7E0EE0EF11C1F5FB3
:1036C0001830E9F62A960FB6F894DEBF0FBECDBFCC
:1036D000DF91CF911F91FF90EF90DF90CF900895F1
:1036E000CF93DF93EC010E94EC1A80916B049091D0
:1036F0006C04019728F4CE01DF91CF910C945F1AEE
:10370000EFE9FFE03197F1F700C00000F2CF0F932F
:103710001F93CF93DF938C01862F65E373E00E94A4
:10372000061F892BC9F4C0913503D0913603209729
:1037300099F0F8018081833069F4CE010E94701BFA
:10374000CE010E94701BCE01DF91CF911F910F918E
:103750000C94701B8430B8F7DF91CF911F910F91BB
:1037600008950F931F93CF93DF938C01EB0165E3D3
:1037700073E08C2F0E94061F892B09F064C0FE01A4
:10378000FF27D8018C91E15CFC4F8130D9F4199668
:103790009C911997992311F080830CC01A969C91E3
:1037A0009923D1F382E0808380913703909138038D
:1037B0000097D9F48091350390913603009709F46E
:1037C00042C013C08230E9F519968C911997811186
:1037D0002DC01A968C9181110EC083E08083809158
:1037E000390390913A03009719F1DF91CF911F911E
:1037F0000F910C94EC1A84E0808380913B039091AC
:103800003C03009791F78091350390913603009720
:10381000F9F00E94701B8091370390913803009754
:1038200021F78091350390913603DFCF85E08083C7
:103830008091350390913603009729F00E94701B08
:10384000F0CF86E08083DF91CF911F910F91089593
:103850008091370390913803B1CF0E94091A0C94DC
:103860001C1BCF92DF92FF920F931F93CF93DF9396
:10387000CDB7DEB72A970FB6F894DEBF0FBECDBF27
:103880008C01603269F5DC011196EC911197EE30F4
:1038900038F5F0E0E65DF94C0C94813588E0ECE118
:1038A000F1E0DE01119601900D928A95E1F780E238
:1038B000F80111928A95E9F784E0D8018C9311966A
:1038C0001C92119712961C92129713961C921397A2
:1038D00088E0FE013196149601900D928A95E1F7E9
:1038E0002A960FB6F894DEBF0FBECDBFDF91CF9101
:1038F0001F910F91FF90DF90CF90089588EFF8010E
:103900008083118212821382EBCF13968C911397CE
:10391000682F70E0762F662712968C91860F972F6E
:10392000911D092E000CAA0BBB0B45E0880F991FB7
:10393000AA1FBB1F4A95D1F7AC01BD01405E5F4F86
:103940006F4F7F4F481759076A077B0748F2883F38
:103950009105A105B10520F6493F510561057105A5
:1039600020F048EF50E060E070E0481B590BBC01CC
:1039700064567E4FC8010E948E35B2CFFC01F280A2
:10398000D38040E06D2D8F2D0E94991E98278927A6
:103990009827D8018D939C9341E06D2D8F2D0E9427
:1039A000991E982789279827F8019383828398CFB7
:1039B00015962D913C91169732272327322714967E
:1039C0004C91149713966C91139712968C910E94B8
:1039D000C41E86CF40E250E06FEF70E00E94AD352C
:1039E00080914D03F801808380914B038183128283
:1039F00082E0838391E09483858372CF81E090E0BD
:103A000090934C0380934B0382E390E090934A039E
:103A1000809349030E94702D90934803809347033D
:103A20005FCF80914B0390914C03892B91F162E021
:103A300080E00E940A14D82E62E081E00E940A14FD
:103A4000F82E80914703909148030E94882D853677
:103A5000910568F1DD2059F1FF2049F10E94702D98
:103A600090934803809347038091490390914A03C0
:103A7000019790934A0380934903892B51F4109244
:103A80004C0310924B0381E090E090934E0380939F
:103A90004D0380914D03D8018C9380914B03119677
:103AA0008C9311978091490312968C9319CF82E3DE
:103AB00090E090934A0380934903EBCF10924E031A
:103AC00010924D030DCF40E250E0BC01FC01828119
:103AD00093810E94752204CFBC016F5F7F4F4FE13D
:103AE00050E012968D919C910E94A722F80180834C
:103AF000F7CEBC016C5F7F4F4CE150E012968D9188
:103B00009C910E94CF22F2CF0E943422E9CE1296DD
:103B10008C911297823009F442C0E8F48823A9F10D
:103B2000813009F0DDCEF80183812AE0F22E9E017A
:103B30002F5F3F4F6901D901EF2D1D92EA95E9F7FB
:103B4000B9010E94061FD8018D93F60101900D92D4
:103B5000FA94E1F7C5CE8330B9F1843009F0C0CED4
:103B600013968C919AE0F8013496DE01119601903B
:103B70000D929A95E1F7BE016F5F7F4F0E94421F41
:103B8000F80180830E941C1BABCE80E2F8011192E9
:103B90008A95E9F788E08C9311968C93A1CE1396C1
:103BA0008C919AE0F8013496DE01119601900D9205
:103BB0009A95E1F7BE016F5F7F4F0E941A1FF801CF
:103BC00080830E94091A8CCE13968C919AE0F92E6C
:103BD000FE0131966F01DF01EF2D1D92EA95E9F7A5
:103BE000B6010E942E1FAFCFAF92BF92CF92DF924D
:103BF000EF92FF920F931F93CF93DF93B82EA62ED1
:103C0000C090B4018091B501C82AC7E0D0E0D12CA2
:103C1000F12CE12CD701C6010C2E04C0B695A79556
:103C2000979587950A94D2F780FF1AC04A2D6B2D7D
:103C30008C2F0E94991E8C018130910589F00E9481
:103C4000EC1AC8010E945F1A81E0DF91CF911F91A9
:103C50000F91FF90EF90DF90CF90BF90AF900895BD
:103C60002197C0F64A2D6B2D80E00E94991EEC0131
:103C70000E94EC1ACE01E6CF84E0089528E0629F0E
:103C8000B001112450E0440F551F640F751F20E14F
:103C9000829FC0011124860F971F879608950F9366
:103CA0001F93CF93DF938430C8F46230B8F444306C
:103CB000A8F40E943E1E8C010E94C435C82FD0E09B
:103CC000DC2FCC27C80101960E94C4359E01282B09
:103CD000C901DF91CF911F910F91089590E080E08D
:103CE000F8CF0F931F93CF93DF93E9018430E0F473
:103CF0006230D0F44430C0F421153C4531F42091B9
:103D00004D0330914E03232B79F00E943E1E8C010F
:103D10006D2F0E94D2356C2FC8010196DF91CF9193
:103D20001F910F910C94D235DF91CF911F910F917C
:103D300008950F931F93CF93DF93843010F5611193
:103D400020C04230F0F424E0829F8001112450E032
:103D5000440F551F040F151F09591F4FC8010E941A
:103D6000C435C82FD0E0DC2FCC27C80101960E94B3
:103D7000C4359E01282BC901DF91CF911F910F916E
:103D8000089590E080E0F8CF0F931F93CF93DF93D7
:103D90008901843028F5611123C0423008F52115CE
:103DA0003C4531F420914D0330914E03232BC1F05B
:103DB00094E0899FE001112450E0440F551FC40F87
:103DC000D51FC959DF4F612FCE010E94D235602F18
:103DD000CE010196DF91CF911F910F910C94D235B6
:103DE000DF91CF911F910F9108958232910520F4B8
:103DF00089589F4F0C94C43580E008958232910514
:103E000020F489589F4F0C94D23508959B01883037
:103E100070F49AE0899FB001112467567F4F4AE001
:103E200050E0C9010E94B43590E080E008958FEF22
:103E30009FEF08959B01883070F49AE0899FB0014C
:103E4000112467567F4F4AE050E0C9010E94F635C1
:103E500090E080E008958FEF9FEF08959B018830F8
:103E600070F49AE0899FB001112467517F4F4AE0B6
:103E700050E0C9010E94B43590E080E008958FEFD2
:103E80009FEF08959B01883070F49AE0899FB001FC
:103E9000112467517F4F4AE050E0C9010E94F63576
:103EA00090E080E008958FEF9FEF08958F929F92AA
:103EB000AF92BF92CF92DF92EF92FF920F931F9338
:103EC000CF93DF93CDB7DEB764970FB6F894DEBF1C
:103ED0000FBECDBFE0904D03F0904E0381E090E027
:103EE00090934E0380934D0384E9C82E82E0D82E30
:103EF0009CEAA92E90E0B92E10E0450100E0F40103
:103F000025913491402F60E0812F0E94711EE2E0E4
:103F10008E0E911C0F5F043091F74501F8E08F0E73
:103F2000911C00E0F40125913491402F61E0812F34
:103F30000E94711E82E0880E911C0F5F043091F781
:103F4000F6012591349140E060E0812F0E94C41E6B
:103F5000F60132962591349141E060E0812F0E9474
:103F6000C41E84E0C80ED11C1F5F90E1A90EB11CD5
:103F7000143009F0C2CF0E9434221C861B861E8694
:103F80001D86188A1F861A8A198A88EC90E09C8BF5
:103F90008B8B10E0BE01655F7F4F812F0E941A1F3F
:103FA0001F5F1830B9F7FE0131966F018AE0119258
:103FB0008A95E9F710E0B601812F0E94421F1F5F2A
:103FC0001830C9F7F0924E03E0924D0364960FB695
:103FD000F894DEBF0FBECDBFDF91CF911F910F913F
:103FE000FF90EF90DF90CF90BF90AF909F908F9019
:103FF0000895EF92FF920F931F93CF93DF93EC01FD
:104000008A017C01E60EF71ECE018796CE15DF05EC
:1040100039F4DF91CF911F910F91FF90EF900895A8
:10402000C034D10540F40E94C435F80180830F5F8D
:104030001F4F2196E9CFF8011082F9CF4F925F927E
:104040006F927F928F929F92AF92BF92CF92DF92A8
:10405000EF92FF920F931F93CF93DF93EC017B01BD
:104060008A0180349105D8F480E490E08C1B9D0B8C
:1040700086179707A0F03E0127E2620E711C80911F
:104080004D0390914E032E01460E571E892BC1F011
:104090007E01C7018796E414F50409F050C0DF9152
:1040A000CF911F910F91FF90EF90DF90CF90BF9035
:1040B000AF909F908F907F906F905F904F900895FA
:1040C0006E0131E0C322DD24C0FF0FC0CE01869611
:1040D0000E94C435F8019081892798278927811586
:1040E0009C4519F48FEFF8018083570140FE13C0FF
:1040F000F1E0AF1AB10848018A0C9B1CC3018E0D78
:104100009F1D0E94C435F401908181159C4519F4CE
:104110008FEFF4018083F801EC0DFD1D2FEFCA1421
:10412000DB0408F0B5CF9081818181159C4511F4A5
:104130002083218382E0C80ED11C3296F0CFE0E4C8
:10414000EE16F10440F4F701EC1BFD0BE00FF11F3C
:1041500060810E94D235FFEFEF1AFF0A9ACF462FF7
:1041600020914B0330914C03232B91F47E3F39F483
:104170006E3F71F480914B0490914C04089584300B
:1041800038F4723028F4643018F4672F0C944F1E02
:1041900090E080E0089580E1089587EC92E0089532
:1041A000EF92FF920F931F93CF93DF93EC018A015D
:1041B0007C01E60EF71ECE01875C9E4FCE15DF0513
:1041C00039F4DF91CF911F910F91FF90EF900895F7
:1041D000C73C22E0D20740F40E94C435F801808336
:1041E0000F5F1F4F2196E7CFF8011082F9CFCF92D2
:1041F000DF92EF92FF920F931F93CF93DF937C0197
:104200006A018C01060F171FEC01CE01875C9E4FDF
:10421000C017D10749F4DF91CF911F910F91FF9003
:10422000EF90DF90CF900895C73C22E0D20740F492
:10423000FE01EE19FF09EC0DFD1D60810E94D235D3
:104240002196E3CFCF93DF93C9E3D1E060E0CE01C5
:104250000E94D2352196C11584E0D807B9F7DF91C5
:10426000CF910895BF92CF92DF92EF92FF920F937A
:104270001F93CF93DF9300D000D0CDB7DEB7F82ED9
:104280002FE0281740F08FEF93E00E94C43509E338
:1042900011E08823D1F00F900F900F900F90DF91D5
:1042A000CF911F910F91FF90EF90DF90CF90BF9033
:1042B0000895011544E0140771F3C8010E94C43544
:1042C000811101C0FA940F5F1F4FF110F2CF1982D4
:1042D0001A821B821C82BB24BA9478015FEFE51A14
:1042E000F50AC8010E94C43589831A82882399F28D
:1042F000813009F047C0680182E0C80ED11CC701B7
:104300000E94C435E82E8A83882329F2C6010E94C0
:10431000C435F82E8FEF8E0D833068F46801E3E02A
:10432000CE0ED11CFB82FF2021F0CE0101960E940F
:104330001E058601D2CFF4E0EF12FBCF680124E026
:10434000C20ED11CC80103960E94C435FF2009F497
:10435000A2CF882309F49FCF8150990BB89E90017A
:10436000B99E300D11244F2D4150550BCA01820FBB
:10437000931F0197F0F2EFE9FFE03197F1F700C0EA
:104380000000F7CFCE0101960E941E056701D1CF34
:10439000EDE4F4E0848195812AE030E0B9010E94E7
:1043A0005935609309018681809308018285809345
:1043B000070184858093060186859785B9010E944F
:1043C0005935609305018089809304018289809327
:1043D0000301848980930201089580914D04909196
:1043E0004E040C94FB2A0F931F93CF93DF930DE49D
:1043F00014E0D0E0C0E0CE010E94F51EF80161910A
:104400008F01861719F0CE010E94FE1E2196C2323E
:10441000D10589F7DF91CF911F910F9108950F93E7
:104420001F93CF93DF930DE414E0D0E0C0E0CE0102
:104430000E94F51EF80181938F012196C232D105A9
:10444000B1F7CAEAD2E0FE0185919491009711F08C
:10445000FC0109952896F3E0C234DF07A1F7DF914C
:10446000CF911F910F910895EDE4F4E0128E138E19
:104470008FEA90E09183808385E0848F88E893E1E0
:10448000938382834CE251E05583448322E330E0FE
:104490003783268385E090E0918780878AE090E0EB
:1044A0009387828764E170E07587648757874687C2
:1044B00044E650E0518B408B48E050E0538B428BF8
:1044C00048E250E0558B448B378B268B28EC30E04C
:1044D000318F208F158E978F868F80E590E091A386
:1044E00080A30E94F3210C940F22EF92FF920F936E
:1044F0001F93CF93DF937C01EB018A016FEF70E094
:10450000CE010E94AD3524EA32E0ACE3B3E090E0A6
:1045100080E0AC014E5F5F4F0417150788F0F9018A
:1045200065917491E616F70630F48C0F9D1FFC011F
:1045300071836083CA01285F3F4FA217B30749F711
:10454000DF91CF911F910F91FF90EF900895DC01C3
:10455000CB0124EA32E0F90165917491A617B707FF
:1045600049F0285F3F4F63E02C333607A1F78FEF08
:104570009FEF0895B9016E5F7F4FFB01A591B49144
:104580004A175B07A0F3FB0145915491F90134965A
:10459000659174910E94A43590E080E00895CF93D6
:1045A000DF93C4EAD2E0FE0125913491821793078C
:1045B00041F0289623E0CC33D207A9F78FEF9FEF85
:1045C0001DC0CE010296FC0125913491421753077C
:1045D000A8F3FC0145915491FE0134968591949184
:1045E0000E94A4350E94F321FE0136968591949194
:1045F000009711F0FC01099590E080E0DF91CF91E8
:1046000008958091650490916604089580916A04EC
:104610008170089580916A048695817008958091D3
:104620006A0482FB882780F9089580916A0483FBDD
:10463000882780F908958091630490916404089517
:10464000AF92BF92CF92DF92EF92FF920F931F93A0
:10465000CF93DF937C015B01C42FD22FFC018281B9
:104660008823F9F0409351030E94702D90935003DA
:1046700080934F0380E28C0F883008F061C0C770D0
:1046800081E001C0880FCA95EAF7DF91CF911F91B1
:104690000F91FF90EF90DF90CF90BF90AF900C9470
:1046A000B30610915103141340C080914F039091B1
:1046B00050030E94882D6C01B701C5010E9401239F
:1046C000C816D90690F5C0E2CD0F1D17B9F080E2EB
:1046D000810F883040F4177081E001C0880F1A956F
:1046E000EAF70E94BA06C83048F481E09D2F97701F
:1046F00001C0880F9A95EAF70E94B306802F0E94A6
:10470000A706C830E8F4D77081E001C0880FDA95B9
:10471000EAF7DF91CF911F910F91FF90EF90DF901B
:10472000CF90BF90AF900C94BA0680E28C0F883087
:1047300038F4C77081E001C0880FCA95EAF7E9CF65
:10474000DF91CF911F910F91FF90EF90DF90CF906D
:10475000BF90AF9008950F939C01CB01233F4CE590
:10476000340759F1A8F4283DFCE53F0701F1293D44
:104770004CE53407D1F1273D3C4591F406E221EEAA
:1047800041EE67ED7CE50E94202380E00F910895C3
:10479000253FFCE53F07E9F0B0F0263F3C45F9F046
:1047A000FC018281882339F110925103EFCF07E297
:1047B00025EE45EE68ED7CE5E6CF06E221EE40EE23
:1047C00063EF7CE5E0CF07E225EE44EE64EF7CE5A5
:1047D000DACF06E221EE42EE65EF7CE5D4CF07E2C8
:1047E00025EE46EE66EF7CE5CECF08E221E045EE11
:1047F00069ED7CE5C8CF81E0C9CFCF93DF93EC01B1
:10480000FB018281882309F419C1C230FCE5DF076E
:10481000C0F1C6319CE5D90730F09E012A5F3C45C6
:104820002930310570F50E9469109093F60380934A
:10483000F503C031ECE5DE0709F4CFC008F05BC03A
:10484000C8308CE5D80709F4B6C088F5C430ECE56B
:10485000DE0709F4A8C0C0F4C2308CE5D80709F41B
:104860009CC08091F5038260C330DC4509F498C098
:104870008091F5039091F6030E9477100E94E5065F
:1048800080E0DF91CF9108958091F5038061C6307B
:10489000ECE5DE0709F484C08091F5038860C73039
:1048A000DC4508F47DC08091F503806279C0CC308E
:1048B0008CE5D80709F489C070F48091F5038C6009
:1048C000CA30ECE5DE0709F46BC008F478C08091CB
:1048D000F5038E7F65C0CE308CE5D80709F479C02A
:1048E0008091F5038B7FCF30DC4508F459C080916F
:1048F000F5038F7E55C0CB3FECE5DE0709F457C0CA
:1049000030F5C3318CE5D80709F46FC078F4C131B4
:10491000ECE5DE0709F465C0C231DC4509F0A8CF3B
:104920000E94E5068091F5038F773AC0C5318CE58A
:10493000D80709F462C008F476C08091F60381605C
:10494000CA3FDC4509F094CF8093F60391CFCF3F67
:10495000FCE5DF0709F44DC088F48091F6038D7FF4
:10496000CD3F9CE5D90781F38091F6038E7FCE3F42
:10497000DC4550F38091F6038360E6CFC130FDE55E
:10498000DF0709F459C008F444C080E0C230DD45B7
:1049900009F06ECF0E94FC106BCF8091F50381600F
:1049A0008093F50365CF8091F5038460F9CF809102
:1049B000F6038260C9CF8091F5038064F1CF0E9435
:1049C000E5068091F5038068EBCF8091F5038D7F3C
:1049D000E7CF8091F503877FE3CF8091F5038F7D4B
:1049E000DFCF8091F5038F7BDBCF8091F503837F51
:1049F000D7CF8091F6038C7FA7CF8091F50382FB00
:104A0000992790F921E0922790FB82F990FB83F996
:104A1000C7CF8091F603982F909591708E7F892B48
:104A200090FB81F991CF0E94E5069091F503892FC3
:104A300097FB87F98058B4CF81E0ACCF81E021CFDC
:104A4000CF93DF93EB0186319C4509F03BC00E9478
:104A5000610F982F9A7A2091670420FF04C0382FA5
:104A6000347409F090E021FF04C0382F317109F04F
:104A700090E022FF04C0382F387809F090E023FF3F
:104A800003C0827209F090E08A81882389F081E076
:104A9000911101C080E08093520389E2911185E376
:104AA0000E94E40E0E94CC0F80E0DF91CF91089528
:104AB00080915203811104C089E20E94EB0EF2CF73
:104AC00085E3FBCF81E0F1CF08950F931F93CF9340
:104AD000DF938091BE03E09153031CE081111AC063
:104AE000DF91CF911F910F91089501E00E0F009378
:104AF0005303CE2FD0E0E19FF0011124E25AFC4F86
:104B000083819481892B29F08081918189238F3F32
:104B1000E9F4E02F8091BE03E81738F31092BE034A
:104B200010925303DDCF18968D919C918F3F98077B
:104B3000D1F061E00E9464251C9FF0011D9FF00DE3
:104B40001124E25AFC4F14821382E3CF1C9FD00140
:104B50001D9FB00D1124A25ABC4F16968D919C91A9
:104B60001797892B01F32081318142815381648120
:104B70007581868197810E94440EDECF1092C0031A
:104B80001092BF0320910B0130910C01EDE4F2E093
:104B900090E080E02817390709F408954581411114
:104BA00002C01482168201963796F4CFDC01609120
:104BB0005C0380915D03962F891301C00895292F0E
:104BC00030E0F901EE0FFF1FEC5AFC4F408151819C
:104BD0004A175B07A1F487E08A9FA0018B9F500DC5
:104BE0001124435B5D4F81E0FA0184839613E6CF85
:104BF0002F5F3F4F2370332720935C0308952F5F6F
:104C00003F4F922F9370D8CF6F927F929F92AF9227
:104C1000BF92CF92DF92EF92FF920F931F93CF93A9
:104C2000DF93DB0114962C911497211169C0A09099
:104C3000BE03EEE5F3E030E020E0B12C662463949F
:104C4000712C2A1508F047C0C284D384ED90FC90E3
:104C500011976FEF7FEF912C492D50E08A01000FE3
:104C6000111F0E0D1F1DE801088119810115110585
:104C700031F0C016D10609F4BA019394EDCF6F3F1D
:104C80007607D1F1E30102C0CC0FDD1F6A95E2F790
:104C9000BC2AB30102C0660F771F9A94E2F7AB01FA
:104CA00041505109B416150629F512964D915C91A3
:104CB00013976CE0629FF001639FF00D1124E25A9C
:104CC000FC4F578346832EEF208321839187808773
:104CD00021E015962C93DF91CF911F910F91FF90BA
:104CE000EF90DF90CF90BF90AF909F907F906F90AC
:104CF0000C94D625148213822F5F3F4F3C96A1CF90
:104D0000DF91CF911F910F91FF90EF90DF90CF90A7
:104D1000BF90AF909F907F906F9008951F93CF9317
:104D2000DF93C0915C0317E080915D038C1307C093
:104D30000E946525DF91CF911F910C94BE25D0E094
:104D4000FE01EE0FFF1FEC5AFC4F80819181189FEE
:104D5000B001199F700D1124635B7D4F0E940426E2
:104D60002196C370E1CF0F931F93CF93DF93DC01A4
:104D70002D913C91119740E090E080E0E82FF0E029
:104D8000EE0FFF1FE20FF31FC081D1812097B9F012
:104D9000FB010081118190E005C0CE17DF0709F407
:104DA00041E09F5FE92FF0E0EE0FFF1FE00FF11FE2
:104DB0000190F081E02D309781F78F5FDFCF4423A2
:104DC00049F0981708F4DB01CD01DF91CF911F91D5
:104DD0000F910895B0E0A0E0F7CF80910A018823F9
:104DE00041F18091C1039091C203009711F10E949B
:104DF000882D2091BF033091C00328173907C8F4CC
:104E000090915C0380915D03981759F00E948E2663
:104E10001092C0031092BF031092C2031092C103FC
:104E200008950E9465251092C2031092C1030C944C
:104E3000BE2508951092C2031092C10310920A0178
:104E400080915D0380935C030E94BE250C946525D0
:104E500080910A0181110C941A2781E080930A0144
:104E600008952F923F924F925F926F927F928F920E
:104E70009F92AF92BF92CF92DF92EF92FF920F93E9
:104E80001F93CF93DF93CDB7DEB72A970FB6F89471
:104E9000DEBF0FBECDBF6C012B01FB011281873F2E
:104EA000FCE59F07F9F4112321F181E080930A01C9
:104EB000812F2A960FB6F894DEBF0FBECDBFDF91CB
:104EC000CF911F910F91FF90EF90DF90CF90BF9007
:104ED000AF909F908F907F906F905F904F903F909A
:104EE0002F900895883F2CE5920709F04DC01111CD
:104EF00048C00DE412E0F12CE12C1986AA24A394F9
:104F0000B12C80910B0190910C01E816F90608F480
:104F100045C0F2018281882309F466C1F985FF2327
:104F200009F462C10E94702D9093C2038093C10363
:104F30008091BE03883008F591E0980F9093BE03EE
:104F400098E0F201DE01119601900D929A95E1F739
:104F50002CE0829FC0011124825A9C4F28E0FE0160
:104F60003196DC0101900D922A95E1F72FEF3FEF8A
:104F7000FC0131872087D386C28611E0F9851F277F
:104F800097CF0E941A2794CF893F9C4509F0B1CF53
:104F9000112309F4AECF0E9428278ACFF80120817F
:104FA000318166246A94762C212C822D90E0FC01BC
:104FB000EE0FFF1FE20FF31F408151814115510594
:104FC00031F0C416D50609F43C012394EECF312C00
:104FD000FFEF6F167F0609F448C0F8014481309056
:104FE0000A01832D411180E0F82FF1703F2EF2016C
:104FF0008281882309F496C0332009F493C0B80154
:10500000C7010E941B234C01F8018581811113C047
:10501000950101C0220F6A94EAF78681822B86836C
:105020008091BF039091C0038815990520F4909258
:10503000C0038092BF03C50102C0880F991F2A9444
:10504000E2F70197F80126812817190671F480917B
:10505000C1039091C203009789F00E94882D8816A1
:10506000990660F421E0F8012483F985F329F98792
:105070002FEFE21AF20A095F1F4F43CF20905C0323
:1050800030915D033A8790E080E0EA852E1215C0EA
:105090008017910751F3822C912CF401EE0FFF1F22
:1050A000EC5AFC4FF182E082FFEF8F1A9F0A23E057
:1050B0008222992480925D03D8CF822C912CF40116
:1050C000EE0FFF1FEC5AFC4F2081318147E0429FD9
:1050D000C001439F900D1124FC01E35BFD4F3F0194
:1050E000B801CF010E94B3260097A9F021E0FC018E
:1050F00024838017910709F4B8CF20915C03221212
:105100000AC06816790639F494012F5F3F4F237067
:10511000332720935C033FEF831A930A482D437093
:10512000242EB3CFF8019580868190E091101EC0A7
:10513000950102C0220F331F2A94E2F72150310952
:105140002817390731F4442309F44CC0C7010E94E1
:10515000D625C50101C0880F6A94EAF7982F90956B
:10516000F801868189238683392C7FCF9C01062C08
:1051700002C0359527950A94E2F7A9014170552799
:10518000BC016150710986239723892B39F5452B82
:1051900029F182819381892BE1F01B821C821D827F
:1051A0001E82FEEFF983FA830E94702D8160582FD2
:1051B0009D838C83F801828193818F8398872981D5
:1051C0003A814B816D817E810E94440EF8011582E7
:1051D000C0CF60E0C7010E946425F8CFF22FF170C4
:1051E0009F2EB7CF932CB5CF90915C0380915D0338
:1051F000981719F00E948E26C0CE0E946525109245
:10520000C2031092C1030E94BE25B7CECF93DF9395
:10521000EC0181E0898B8F810E94640F88850E9458
:10522000770F0E94CC0FEA81FB81309739F06C89AF
:105230007D89CE010696DF91CF910994DF91CF91C0
:105240000895EF92FF920F931F93CF93DF93EC019A
:105250008A85811134C0EB80FC8087E5F81A26E14D
:105260002E9DC0012F9D900D1124DC01AB57BD4F29
:105270001496ED91FC911597309731F054966D91FD
:105280007C9185579D4F099586E18E9D80018F9D6C
:10529000100D11240B571D4FF80187810E946A0FD2
:1052A000F80180850E947D0F0E94CC0F188219861C
:1052B0001B861E821D821092C4031092C303DF91CD
:1052C000CF911F910F91FF90EF900895DF92EF9291
:1052D000FF920F931F93CF93DF937C01FB01828199
:1052E000882391F080910D018F3F71F0C5E8D2E0E5
:1052F00010E000E0DD24D39480910D01082E000C15
:10530000990B8017910744F4DF91CF911F910F9172
:10531000FF90EF90DF9008958E818823D9F08985E2
:105320009A858E159F0539F48091C3039091C4032B
:105330008E159F0579F0DF86FC86EB8689898111C1
:1053400003C0CE010E940629CE0106960E942129A3
:105350000E94840F0F5F1F4F6696CECFEF92FF9291
:105360000F931F93CF93DF937C0197558F3F910548
:1053700009F0D8F520910D01022E000C330B2817EF
:10538000390714F480930D01FB01228136E1389F27
:105390008001399F100D1124E801CB57DD4F288B78
:1053A00092818E81992349F1FA86E9868F5F8E83F7
:1053B0000E94702D9E878D870E948A0F8F830E9486
:1053C000610F88870E94740F9885892B8887E881F0
:1053D000F981309731F06C897D89C80185579D4FDF
:1053E0000995F092C403E092C30381E0DF91CF916D
:1053F0001F910F91FF90EF9008958823B1F3898951
:10540000882399F3C80185579D4F0E942129EDCF2C
:10541000CF92DF92EF92FF920F931F93CF93DF9380
:1054200080910D0110E006E18F3FF1F5DF91CF9102
:105430001F910F91FF90EF90DF90CF9008950E9DF8
:10544000F0010F9DF00D1124EB57FD4FC288D3885A
:10545000C114D10439F470E060E0818592850E9426
:1054600001236C010E9DE0010F9DD00D1124CB573F
:10547000DD4F8E818823B9F08D859E850E94882D11
:10548000C816D90680F4109F7001112489898111F2
:1054900005C0C7018B579D4F0E940629C70185573C
:1054A0009D4F0E9421291F5FE12EF12C80910D015B
:1054B000082E000C990B8E159F050CF6B7CFFF92A6
:1054C0000F931F93CF93DF938C01EB01F42E809108
:1054D0000E0182FF4AC08B7F80930E018091C7032B
:1054E0009091C8039B01281B390BC90120910F0122
:1054F0003091100182179307B8F48091C5030E9480
:10550000A80580910E018D7F80930E0180916B0420
:1055100090916C04019710F58091C5030E943A06A2
:1055200082E00E947D0F2BC082E00E94770F809165
:10553000C5030E94A80580910E01826080930E0130
:105540008091680485FFE2CF86FDE0CFFF20F1F275
:10555000DF91CF911F910F91FF900895EFE9FFE048
:105560003197F1F700C00000D5CF802F0E943A0696
:105570008091C5039091C6038017910789F20E941C
:10558000CC0FD093C803C093C703E2CF80916804C7
:1055900080FF1DC080910E0182FF19C00E94702DF6
:1055A0002091C7033091C803AC01421B530B9A01F1
:1055B00040910F01509110012417350740F041E050
:1055C000BC018091C5039091C6030C945F2A089595
:1055D00090910E01892F8E7F90FF816080930E0144
:1055E00082E00C947D0F80910E018E7F80930E01DE
:1055F00082E00C947D0F9093100180930F01089529
:105600008832910538F48E319105E8F40497A0F4BE
:1056100080E008958933910558F48D32910510F496
:105620008B97B1F78091680482FB882780F908C0C6
:1056300084369105B9F3ECCF80916804829581702E
:1056400091E0892708958091680483FB882780F979
:10565000F7CFCF92DF92EF92FF920F931F93CF93EA
:105660008C016B018091680480FD0AC0C1E08C2F21
:10567000CF911F910F91FF90EF90DF90CF90089501
:105680000E94702D7C01F601C281CC2329F180910A
:105690000E0182FF06C040E0B70190E080E00E946A
:1056A0005F2A82E00E947D0F0B31FCE51F0759F055
:1056B0000C314CE5140769F00A315CE5150761F41B
:1056C0000E94E82AD4CF80910E01816080930E0160
:1056D000CECF0E94F32ACBCFB601C8010E94002B87
:1056E000882321F2F601C281CC2309F44EC08091B7
:1056F0000E0180FFBBCF8091680481FF15C08091AF
:10570000680485FD16C01093C6030093C503F0928C
:10571000C803E092C70380910E01846080930E015C
:1057200082E00E9434102FC00E94610F882339F359
:105730009DCF2091C7033091C803A701421B530B93
:105740009A0186FD04C080910E0181FDDCCF283CCA
:105750003105C8F68091C5039091C6030817190753
:1057600091F680910E0181FBCC27C0F981FD04C028
:10577000802F0E94A8057BCF82E00E94770F809146
:10578000C5030E94A805C0E072CF40E0B701C80180
:105790000E945F2A6CCF9093CE038093CD0308952F
:1057A000E091CD03F091CE03309721F00190F0818C
:1057B000E02D099480E00895E091CD03F091CE03AF
:1057C000309799F020911B01222359F02091F50385
:1057D00027FF07C0DC012C9111962C93119725E02F
:1057E0002C930280F381E02D09940895E091CD037C
:1057F000F091CE03309739F022E0DC012C93048045
:10580000F581E02D099408952091CB033091CC03CC
:105810002817390771F09093CC038093CB03E09164
:10582000CD03F091CE03309721F00680F781E02D73
:10583000099408952091C9033091CA0328173907A4
:1058400071F09093CA038093C903E091CD03F09166
:10585000CE03309721F00084F185E02D099408955E
:10586000FC01329680911B01882321F08091F50381
:105870009EE187FF96E080E0915008F40895219121
:105880002223D1F38F5FF8CF662301F120911B0112
:105890002223F1F02091F50327FF1AC0462F4695E9
:1058A000469546954E3190F4677021E030E002C095
:1058B000220F331F6A95E2F7840F911DFC0182814C
:1058C00090E02823392381E0232B69F480E00895B8
:1058D000FC01329608962191261721F0E817F90766
:1058E000D1F7F4CF81E008959C01FC0132969FEF3F
:1058F00080E04191461751F09F3F19F4411101C0DA
:10590000982F8F5F8630A9F79F3F09F40895290FDC
:10591000311D97FD3A95F90162830895FC01329695
:1059200008962191261303C0DF0111971C92E817F6
:10593000F907B9F70895E62FE695E695E695EE3175
:1059400068F4E80FF92FF11D677021E030E001C025
:10595000220F6A95EAF78281822B82830895E62FCF
:10596000E695E695E695EE3170F4E80FF92FF11D16
:10597000677021E030E001C0220F6A95EAF72095B8
:10598000828128232283089520911B01222329F05C
:105990002091F50327FD0C949B2C0C94742C2091E2
:1059A0001B01222329F02091F50327FD0C94AF2C35
:1059B0000C948E2CFC01329680911B01882351F0AF
:1059C0008091F50387FF06C08EE1DF011D928A9565
:1059D000E9F7089586E0F9CF0895089508950C94A5
:1059E000EE2C80917704843049F10E94EF2C80E006
:1059F0000E9429051092CF0388E190E020E40FB6C1
:105A0000F894A895809360000FBE2093600083B740
:105A1000817F846083BF83B7816083BF78948895DA
:105A200083B78E7F83BF0FB6F894A89580916000EE
:105A3000886180936000109260000FBE0895089501
:105A40000E94ED2C0E94D1140E941F2D80E00E9424
:105A50001E1491E0811107C081E00E941E1491E0A4
:105A6000811101C090E0892F089508950C94352D7F
:105A70000E94E5060E94D02B0E9429050C94362D29
:105A80001F921FB61F9211248F939F93AF93BF93C2
:105A90008091CF03811113C080916F0490917004A5
:105AA000A0917104B09172044196A11DB11D809323
:105AB0006F0490937004A0937104B0937204BF912B
:105AC000AF919F918F911F901FBE1F90189582E0FC
:105AD00084BD93E095BD9AEF97BD80936E000895C5
:105AE0002FB7F89480916F0490917004A091710485
:105AF000B09172042FBF08952FB7F89460916F048E
:105B00007091700480917104909172042FBF089578
:105B10009C014FB7F89480916F0490917004A0910C
:105B20007104B09172044FBF821B930B0895789457
:105B30001F921FB61F9211248F939F93AF93BF9311
:105B400080916F0490917004A0917104B0917204DF
:105B50000196A11DB11D80936F0490937004A093D2
:105B60007104B0937204BF91AF919F918F911F9078
:105B70001FBE1F90189581E08093E00080E2809323
:105B8000D8001092C9008FE19EE40197F1F700C0A0
:105B9000000087E090EBDC01809380049093810407
:105BA000A0938204B093830488E19CE00FB6F8943C
:105BB000A895809360000FBE90936000FFCF9093F4
:105BC000AD018093AC0108958091F3030895909105
:105BD0007704943029F58093D0037093D2036093B7
:105BE000D1039093E9008FEF9091E800815095FDEB
:105BF00006C095ED9A95F1F700008111F5CF8091DF
:105C0000E80085FF0DC050E040E063E070E080ED0B
:105C100093E00E9479308091E8008E778093E800CD
:105C20000895BC0184E00C94E72DBC0183E00C9442
:105C3000E72D9C0184E08093E9009FEF8091E800CC
:105C4000915085FD06C085ED8A95F1F70000911110
:105C5000F5CF8091E80085FF0CC050E040E066E0A1
:105C600070E0C9010E9479308091E8008E778093BE
:105C7000E8000895CF93DF93EC0180911B01882306
:105C8000B1F18091F50387FF32C060E284E0809338
:105C9000E9008FEF9091E800815095FD06C095EDE9
:105CA0009A95F1F700008111F5CF8091E80085FF0A
:105CB0001BC080911B0170E050E040E0811104C0E6
:105CC00050E040E068E070E0CE010E9479308091C1
:105CD000E8008E778093E80080E2FE01A3EDB3E058
:105CE00001900D928A95E1F7DF91CF91089568E0D8
:105CF00081E0CDCFCF93FC01603221F58091770414
:105D0000843001F5C091E900CF702091EC00922F12
:105D1000917020FD90E8C92B82E08093E90080918A
:105D2000E80080FF0CC050E040E060E270E0CF018E
:105D30000E9479308091E8008E778093E800CF70E0
:105D4000C093E900CF91089580917604811109C034
:105D50000E9458320E94B5328091E20084608093A4
:105D6000E200089510927604089508950895089524
:105D700042E061EC81E00E94D43142E261EC84E0D7
:105D80000E94D43142E261EC82E00E94D43142E2CE
:105D900060EC83E00C94D43180917904833009F471
:105DA00061C030F48130D1F1823009F49DC0089592
:105DB0008A3009F489C08B3009F46FC0893009F04A
:105DC00050C080917804813209F04BC080917C04EE
:105DD00090917D04009719F0029709F042C08091DC
:105DE000E800877F8093E8008091E80082FF35C05B
:105DF0009091F3008091F200029729F48091F100D4
:105E00008B7F813021F48091F1008093F3038091A6
:105E1000E8008B778093E8000C9408328091780436
:105E2000813AF9F48091E800877F8093E8008091BF
:105E30007C0490917D04892B61F460E283ED93E012
:105E400070E00E9417318091E8008B778093E80022
:105E5000089560E090E080E0F3CF809177048111B5
:105E6000C3CF089580917804813AD9F780917C045A
:105E700090917D04892BA9F78091E800877F80931A
:105E8000E8008091E80080FFFCCF80911B018093A7
:105E9000F1008091E8008E77BDCF80917804813247
:105EA00001F780917C0490917D04892BD1F680913B
:105EB000E800877F8093E8000E94083280917A048E
:105EC00080931B010C94E50680917804813249F699
:105ED0008091E800877F8093E8000E9408328091DB
:105EE0007B048093F403089580917804813A09F04B
:105EF000B8CF8091E800877F8093E8008091E80028
:105F000080FFFCCF8091F403C2CF84B7877F84BF2A
:105F10000FB6F894A8958091600088618093600026
:105F2000109260000FBE80E890E00FB6F894809366
:105F30006100909361000FBE0C9435110E9458329D
:105F40000E94B532E2EEF0E0808184608083789434
:105F50000E943E350E944D1181E191E00C94CB2BC3
:105F6000CF93DF93CDB7DEB7A0970FB6F894DEBF1F
:105F70000FBECDBF80917704853031F480917704D6
:105F8000853091F10E94382D0E945711809177043D
:105F9000843009F583E08093E9008091E80082FF76
:105FA0001AC08091E80090E085FF09C050E040E011
:105FB00060E270E0CE0101960E94C83091E08091CD
:105FC000E8008B778093E800992329F060E2CE0106
:105FD00001960E94F318A0960FB6F894DEBF0FBE8C
:105FE000CDBFDF91CF9108950E94F12C809175046F
:105FF000882321F20E94202D882309F4BFCF0E941C
:1060000063300E94E506BACF0C940630292F33275F
:106010002330310521F168F42130310509F449C0FC
:106020002230310509F44AC090E080E030E020E001
:1060300029C02132310581F122323105A9F76330BF
:10604000710590F7FB01EE0FFF1FE156FE4F208117
:10605000318164567E4FFB01808190E013C0992707
:106060008130910599F0009741F08230910589F0D7
:106070000397D1F6ECE3F3E002C0E4E9F3E08491A6
:1060800090E09F01FA01318320830895EEE7F3E069
:10609000F6CFEAE5F3E0F3CF6330710528F6660F3B
:1060A000771FFB01EB55FE4F2081318189E090E0A5
:1060B000E9CF82E190E023EF33E0E4CF8BE590E09D
:1060C00028E933E0DFCF80E189BD82E189BD09B4F1
:1060D00000FEFDCF8091D8008F7D8093D800809105
:1060E000E00082608093E0008091E00081FDFCCFC1
:1060F0000895AF92BF92CF92DF92FF920F931F93BA
:10610000CF93DF936C01EB018A010E942732F82EB6
:10611000811123C00115110539F0F80180819181A9
:10612000C81BD90BC80ED91EB12CA12C2097A9F0E1
:106130008091E80085FD22C08091E8008E778093F1
:10614000E80001151105A1F0F80180819181A80EE8
:10615000B91EB182A08285E0F82E8F2DDF91CF91FC
:106160001F910F91FF90DF90CF90BF90AF90089557
:106170000E9427328823D1F2F82EEFCFF6018191C9
:106180006F018093F1002197FFEFAF1ABF0ACECFC6
:10619000AF92BF92CF92DF92FF920F931F93CF9354
:1061A000DF936C01EB018A010E942732F82E8111E6
:1061B00023C00115110539F0F80180819181C81BB8
:1061C000D90BC80ED91EB12CA12C2097A9F0809113
:1061D000E80085FD22C08091E8008B778093E8007D
:1061E00001151105A1F0F80180819181A80EB91E59
:1061F000B182A08285E0F82E8F2DDF91CF911F9183
:106200000F91FF90DF90CF90BF90AF9008950E94C4
:1062100027328823D1F2F82EEFCF8091F100F601DA
:1062200081936F012197FFEFAF1ABF0ACECFFC0118
:1062300080917E0490917F0486179707A0F06115E6
:10624000710529F49091E8009E779093E80090E022
:106250006115710551F4911108C08091E80082FF29
:1062600034C080E00895BC01F2CF80917704882388
:10627000C1F18530C1F18091E80083FD30C080918B
:10628000E80082FDEACF8091E80080FFE1CF8091B5
:10629000F3002091F200382F6115710519F02830B4
:1062A000310558F091E02830310509F090E0209157
:1062B000E8002E772093E800CBCF81918093F10006
:1062C000615071092F5F3F4FE7CF8091770488239A
:1062D00041F0853041F08091E80083FFBECF81E03E
:1062E000089582E0089583E00895FC0180917E0482
:1062F00090917F0486179707A0F06115710529F426
:106300008091E8008E778093E80090E06115710538
:1063100051F4911108C08091E80082FF35C080E0FF
:106320000895BC01F2CF809177048823C9F18530AC
:10633000C9F18091E80083FD31C08091E80082FDC1
:10634000EACF8091E80080FFE1CF8091F3002091B7
:10635000F200382F6115710519F02830310558F019
:1063600091E02830310509F090E08091E8008E77C7
:106370008093E800CBCF84918093F10031966150F7
:1063800071092F5F3F4FE6CF80917704882341F05A
:10639000853041F08091E80083FFBDCF81E0089512
:1063A00082E0089583E00895982F973028F08F7049
:1063B0008093E90081E008959093E900242F762FDF
:1063C00050E0981731F07091EC002091ED00509161
:1063D000F00021FD02C09F5FE8CF3091EB003E7FCF
:1063E0003093EB003091ED003D7F3093ED00309124
:1063F000EB0031603093EB007093EC002093ED00E4
:106400005093F0002091EE0027FDE5CF80E0089545
:106410008091780487FF13C08091E80082FF06C056
:106420008091E8008B778093E80004C08091770426
:106430008111F2CF0895809177048823D9F3809158
:10644000E80080FFF8CF8091E8008E77ECCF2091B4
:10645000E4003091E50095E6A9012091EC00822F3F
:10646000817020FF06C08091E80080FF06C080E0B8
:1064700008952091E80022FD1AC0809177048823B6
:1064800089F0853089F08091EB0085FD0FC0209167
:10649000E4003091E50042175307F9F29150E1F61C
:1064A00084E0089582E0089583E0089581E00895EE
:1064B0000E94C6320E94CE32E0EEF0E08081816020
:1064C0008083E8EDF0E080818F77808319BCA7EDB1
:1064D000B0E08C918E7F8C9380818F7E8083109230
:1064E000760408950F931F93CF93DF930E94C632D3
:1064F0000E94CE32C8EDD0E088818F778883888172
:106500008068888388818F7D888319BC1092770486
:1065100010927304109275041092740400EE10E04F
:10652000F80180818B7F808388818160888342E04D
:1065300060E080E00E94D431E1EEF0E080818E7F67
:106540008083E2EEF0E080818160808380818860DA
:106550008083F80180818E7F808388818061888339
:10656000DF91CF911F910F910895E8EDF0E08081C8
:106570008F7E8083E7EDF0E080818160808384E01E
:1065800082BF81E0809376040C947232E8EDF0E0F3
:1065900080818E7F80831092E20008951092DA004D
:1065A0001092E10008951F920F920FB60F921124DE
:1065B0002F933F934F935F936F937F938F939F930B
:1065C000AF93BF93EF93FF938091E10082FF0BC0E5
:1065D0008091E20082FF07C08091E1008B7F809371
:1065E000E1000E943D358091DA0080FF19C0809162
:1065F000D80080FF15C08091DA008E7F8093DA008A
:106600008091D90080FF96C080E189BD82E189BD7B
:1066100009B400FEFDCF81E0809377040E94A42E90
:106620008091E10080FF19C08091E20080FF15C0D9
:106630008091E2008E7F8093E2008091E200806191
:106640008093E2008091D80080628093D80019BCCA
:1066500085E0809377040E94B62E8091E10084FF4C
:106660002BC08091E20084FF27C080E189BD82E1D8
:1066700089BD89B5982F917080FFFBCF8091D8009C
:106680008F7D8093D8008091E1008F7E8093E10020
:106690008091E2008F7E8093E2008091E200816031
:1066A0008093E20080917304882309F449C084E058
:1066B000809377040E94B72E8091E10083FF29C068
:1066C0008091E20083FF25C08091E100877F809365
:1066D000E10082E080937704109273048091E100DE
:1066E0008E7F8093E1008091E2008E7F8093E200B4
:1066F0008091E20080618093E20042E060E080E00F
:106700000E94D4318091F00088608093F0000E9454
:10671000B52EFF91EF91BF91AF919F918F917F9196
:106720006F915F914F913F912F910F900FBE0F90FE
:106730001F90189519BC109277040E94B22E70CF4A
:106740008091E30087FD93E090937704B3CF1F928D
:106750000F920FB60F9211242F933F934F935F9395
:106760006F937F938F939F93AF93BF93CF93DF9359
:10677000EF93FF93D091E900DF708091EC00C82F78
:10678000C17080FDC0E81092E9008091F000877F21
:106790008093F00078940E94EB331092E90080918E
:1067A000F00088608093F000CD2BCF70C093E9009B
:1067B000FF91EF91DF91CF91BF91AF919F918F9119
:1067C0007F916F915F914F913F912F910F900FBEED
:1067D0000F901F9018951F93CF93DF93CDB7DEB71F
:1067E000AA970FB6F894DEBF0FBECDBF88E794E03E
:1067F0002091F100FC012193CF01F4E080389F0744
:10680000B9F70E94CC2E8091E80083FF1EC18091D1
:106810007804909179049A3008F017C1E92FF0E0DC
:10682000E85CF94C0C948135803899F0823809F095
:106830000CC180917C048F70873008F006C1809372
:10684000E9008091EB0085FB882780F91092E90030
:1068500006C08091740490917504911182609091AA
:10686000E800977F9093E8008093F1001092F10088
:106870008091E8008E77E5C0882309F4D3C0823088
:1068800009F0E3C080917A048111D6C080917C0424
:106890008F702FEF280F263008F0D7C08093E900C3
:1068A0002091EB0020FFC8C0933031F48091EB00C1
:1068B00080628093EB00C0C09091EB009061909358
:1068C000EB0021E030E001C0220F8A95EAF7209327
:1068D000EA001092EA008091EB008860EACF811113
:1068E000B4C010917A041F778091E3008078812BE7
:1068F0008093E3008091E800877F8093E8000E9406
:1069000008328091E80080FFFCCF8091E30080682E
:106910008093E30082E0111183E08093770495C0B7
:106920008058823008F091C080917A0490917B0465
:106930008C3D23E09207A1F583E08A838AE2898374
:106940004FB7F894DE01139620E03EE051E2E32FCA
:10695000F0E050935700E49120FF03C0E295EF7000
:106960003F5FEF708E2F90E0EA30C0F0C7968D93B6
:106970009D932F5F243159F74FBF8091E800877FA7
:106980008093E8006AE270E0CE0101960E94173120
:106990008091E8008B778093E80057C0C096E7CFDE
:1069A00060917C0470917D04AE014F5F5F4F0E9447
:1069B0000430BC01892B09F448C09091E800977F0E
:1069C0009093E80089819A810E947531E1CF8038E7
:1069D000E1F58091E800877F8093E800809173045F
:1069E0008093F10045CF811130C090917A049230AC
:1069F00060F58091E800877F8093E80090937304AE
:106A00000E94083280917304882311F084E005C04D
:106A10008091E30087FDFACF81E0809377040E94A4
:106A2000B82E13C080917A04813079F481E09330DC
:106A300009F080E0809375041092E9008091E800ED
:106A4000877F8093E8000E9408328091E80083FFEE
:106A50000AC08091E800877F8093E8008091EB0076
:106A600080628093EB00AA960FB6F894DEBF0FBE4B
:106A7000CDBFDF91CF911F9108950895CF9380915D
:106A800077048823A1F0C091E900CF709091EC00C9
:106A9000892F817090FD80E8C82B1092E9008091C9
:106AA000E80083FD0E94EB33CF70C093E900CF91E3
:106AB0000895AA1BBB1B51E107C0AA1FBB1FA61745
:106AC000B70710F0A61BB70B881F991F5A95A9F797
:106AD00080959095BC01CD01089597FB072E16F483
:106AE000009407D077FD09D00E94593507FC05D0E6
:106AF0003EF4909581959F4F0895709561957F4FD5
:106B00000895EE0FFF1F0590F491E02D0994692779
:106B1000962769277827872778270895FB01DC01C6
:106B200002C005900D9241505040D8F70895FB01E6
:106B3000DC0104C08D910190801921F44150504036
:106B4000C8F7881B990B0895FB01DC0102C0019076
:106B50000D9241505040D8F70895DC0101C06D936B
:106B600041505040E0F70895DC01CB01FC01F99958
:106B7000FECF06C0F2BDE1BDF89A319600B40D9289
:106B800041505040B8F70895F999FECF92BD81BDAC
:106B9000F89A992780B50895A8E1B0E042E050E066
:106BA0000C94B635262FF999FECF92BD81BDF89A87
:106BB000019700B4021639F01FBA20BD0FB6F89441
:106BC000FA9AF99A0FBE08950396272F0E94D3359B
:106BD0000E94D235252F0E94D335242F0C94D33513
:106BE0000196272F0E94D3350C94D235DC01CB01BE
:106BF00003C02D910E94013641505040D0F70895B6
:106C0000262FF999FECF1FBA92BD81BD20BD0FB6C8
:106C1000F894FA9AF99A0FBE01960895F894FFCF66
:106C2000F406F406FD06FD06FF06FD06FD06FD065C
:106C3000F406F4060407FD06FD0604074C074C079E
:106C4000AF07AF072F0849087C077C075608BF0825
:106C5000D008D0084E1C7E1C851CBE1CD81CEA1C0B
:106C6000FE1C111D5E1D631D6C1D791D841D871D7D
:106C700014343C3425353C3425356F349034253577
:046C8000E734F334CE
:106C840007022808641E140A321E010800FF01AF1F
:106C940000E42D3A2E192E152E112E01A745215D43
:106CA400F47B2967E200E900EA00B500B600B7000A
:106CB400CD008301CC008A019201940121022302B8
:106CC40024022502260227022A02B300B4006F0020
:106CD4007000818283E200E900EA00B500B600B7E3
:106CE40000CD008301CC008A01920194012102238A
:106CF4000224022502260227022A02B300B4006FEE
:106D040000700081828336666794353400FF010089
:106D1400010000FFFF0000010001FF004022BCE36E
:0C6D24000405042704AA03C303E30300D2
:00000001FF
